S01B00006F70656E626C745F656B5F6C6D3373363936352E737265632E
S113000098180020C97B00000D7C00000D7C0000C6
S11300100D7C00000D7C00000D7C00000D7C0000B8
S11300200D7C00000D7C00000D7C00000D7C0000A8
S11300300D7C00000D7C00000D7C00000D7C000098
S11300400D7C00000D7C00000D7C00000D7C000088
S11300500D7C00000D7C00000D7C00000D7C000078
S11300600D7C00000D7C00000D7C00000D7C000068
S11300700D7C00000D7C00000D7C00000D7C000058
S11300800D7C00000D7C00000D7C00000D7C000048
S11300900D7C00000D7C00000D7C00000D7C000038
S11300A00D7C00000D7C00000D7C00000D7C000028
S11300B00D7C00000D7C00000D7C00000D7C000018
S11300C00D7C00000D7C00000D7C00000D7C000008
S11300D00D7C00000D7C00000D7C00000D7C0000F8
S11300E00D7C00000D7C00000D7C00000D7C0000E8
S11300F003E00B780370491C401C13005A1E002BAC
S1130100F7D1704701E00170401C13005A1E002B08
S1130110F9D1704710B400231400621E002C06D0DD
S113012003780C781B1B491C401C002BF4D01800CE
S113013010BC704700E0401C0278002A02D002780C
S11301408A42F8D10078704770B5040020790028FD
S113015023D0256B01232A0014F13401607802F0C6
S1130160E3F9002801D0012018E000202071606A22
S1130170854212D3606AE169081885420DD2E67897
S113018009E0E069451901232A0014F1340160787B
S113019002F0CAF9761E022EF3D2002070BD38B5E3
S11301A004000D00206B854212D02000FFF7CCFF25
S11301B0002801D001200CE001232A0014F13401AD
S11301C0607802F064F9002801D0012001E0256381
S11301D0002032BD38B504002000FFF7B5FF05004C
S11301E0EDB2002D5DD12078032852D1607900282A
S11301F04FD0002020634FF40072002114F134002A
S1130200FFF780FF552084F83202AA2084F83302D5
S1130210522084F83400522084F83500612084F898
S11302203600412084F83700722084F818027220C6
S113023084F81902412084F81A02612084F81B0210
S1130240206984F81C02206980B2000A84F81D0227
S11302502069000C84F81E022069000E84F81F0235
S1130260E06884F82002E06880B2000A84F8210281
S1130270E068000C84F82202E068000E84F823028F
S11302800123626914F13401607802F04DF9002011
S1130290607100220021607802F0A4F9002800D0E7
S11302A001252800C0B232BD891E8269921E914286
S11302B001D3002003E08278C06A02FB010070478A
S11302C0F8B504000D00022D02D3A069854201D3C4
S11302D0012014E02078012804D00ED303284AD04A
S11302E032D30AE02E0016EB5606606A10EB562154
S11302F02000FFF754FF002802D05FF0FF30F2BD6A
S11303004FF40070B6FBF0F101FB1061081990F88E
S11303103470761C606A10EB56212000FFF73FFF13
S11303200028EAD14FF40070B6FBF0F101FB106134
S1130330081990F8340057EA0027E80701D538096E
S113034001E03805000DDAE7606A10EB15212000A2
S1130350FFF725FF0028D0D168004FF40071B0FBEF
S1130360F1F202FB1102101934304178007850EA9E
S1130370012080B2C3E7606A10EBD5112000FFF7BB
S11303800EFF0028B9D1A8004FF40071B0FBF1F2C0
S113039002FB110210193430C1788278120452EA37
S11303A00161427851EA0221007808430001000902
S11303B0A5E7F8B504000D001600022D02D3A069CC
S11303C0854201D3022082E02078012804D07BD327
S11303D0032858D040D377E02F0017EB5707606A03
S11303E010EB57212000FFF7DAFEC0B200286CD1D1
S11303F04FF40070B7FBF0F101FB1071081910F114
S11304003401E80705D5087810F00F0050EA06100B
S113041000E0300008707F1C01202071606A10EB3E
S113042057212000FFF7BBFEC0B200284DD14FF486
S11304300071B7FBF1F202FB117211193431EA07B2
S113044001D5320906E00A7812F0F002330A13F0FB
S11304500F031A430A7038E0606A10EB152120007C
S1130460FFF79DFEC0B200282FD169004FF400723F
S1130470B1FBF2F303FB1213191934310E70B6B247
S1130480320A4A7021E0606A10EBD5112000FFF7B0
S113049086FEC0B2002818D1A9004FF40072B1FB47
S11304A0F2F303FB121319193431CA78120612F04D
S11304B0704216430E70320092B2120A4A70320C25
S11304C08A70320ECA7000E0022001212171C0B28C
S11304D0F2BDF8B504000E00022E02D3A0698642D4
S11304E001D3022527E0002509E0206910F1010F5E
S11304F004D02069401C2061012060713E00A06985
S1130500864218D231002000FFF7DAFE0700002FE0
S113051011D0012F01D102250DE017F1010F01D1F6
S1130520012508E0002231002000FFF742FF05000A
S1130530EDB2002DD9D02800C0B2F2BDF8B5040048
S11305400E00002E07D1E768002F02D0A069874271
S11305500DD301270BE031002000FFF7B1FE022884
S113056001D2012043E0A169884240D337003D0015
S11305706D1CA069854204D30225AF4201D200203C
S113058035E029002000FFF79BFE00281DD17FF0F5
S1130590704229002000FFF70CFFC0B2002806D1EA
S11305A0002E04D02A0031002000FFF702FFC0B261
S11305B0002814D1E560206910F1010F16D02069DC
S11305C0401E20610120607110E010F1010F01D084
S11305D0012800D10BE0BD42CAD1002007E0C0B21F
S11305E0012802D15FF0FF3500E001252800F2BDAB
S11305F070B504000D00E580A068012803D02168CF
S11306008969884201D3022048E0002805D1216885
S11306100978032901D12068806A00280ED1E0609E
S113062020680089ADB2854201D3022036E02068FB
S1130630806AADB210EB1510206123E0216889783F
S113064089B20E0100E0AD1BADB2B6B2B54210D313
S113065001002068FFF734FE10F1010F01D10120E1
S11306601CE0022803D3216889698842EBD3022065
S113067014E0E06001002068FFF716FEADB210EB55
S113068015102061ADB21020B5FBF0F101FB105143
S1130690206810EB411034306061002070BDF8B563
S11306A004000D00E088461CB6B2002E02D020697A
S11306B0002801D1042087E0B6B21020B6FBF0F187
S11306C001FB1061002972D12069401C2061E0689F
S11306D0002806D120680089B6B2864267D3042078
S11306E072E0B6B220688078401E10EA161F5ED110
S11306F0E1682068FFF7E4FD0700022F01D2022021
S113070062E017F1010F01D101205DE020688069EA
S1130710874246D3002D01D1042055E0E1682068CA
S1130720FFF70CFF0700002F01D107204CE0012F39
S113073001D1022048E017F1010F01D1012043E06B
S11307402068FFF701FD002801D001203CE04FF4B0
S11307500072002120683430FFF7D4FC390020688F
S1130760FFF7A2FD21680863002505E02068006BFF
S1130770401C216808636D1C20688078EDB28542B6
S113078009D22068012101712068FFF7DDFC0028EF
S1130790ECD0012018E02068006BEDB2401B21680A
S11307A00863E76039002068FFF77EFD2061E6807A
S11307B0B6B21020B6FBF0F101FB1061206810EB1B
S11307C04110343060610020F2BD70B504000D00AA
S11307D000212000FFF70CFFC0B200281BD1002627
S11307E021692068FFF7DBFCC0B2002813D16169DE
S11307F00978E52903D061690978002903D1761CB9
S1130800AE4201D107E0002601212000FFF747FF97
S1130810C0B20028E4D0C0B270BDCA7E8B7E53EA59
S1130820022292B20078032806D1487D097D51EA5C
S1130830002080B252EA00421000704781760A001C
S113084092B2120AC2760A0C0275090C89B2090A1C
S1130850417570472DE9F04104000D00287830F00F
S11308604000401E0D2101FB00F600275FF0010847
S1130870DFF8180D385C40194078DFF8101D795CFA
S1130880495D51EA00201FFA88F8B8F1000F11D031
S113089080B202F00CF88046FF2E09D234F816001C
S11308A002F005F8761C1FFA88F880B2804508D05B
S11308B0002018E080B24FF6FF71884201D000207A
S11308C011E07F1C0D2FD3D3287840060AD51FFAD8
S11308D088F8B8F1000F05D034F81600002801D0CC
S11308E0002000E00120BDE8F08170B40A7812F025
S11308F03F02521E0D235A4300230124DFF88C5C6F
S11309005D5D6D186D78DFF8846C9E5D765C56EAEB
S11309100525A4B2002C11D0FF2A01D3002018E031
S11309202C0020F81240521C5B1C0D2BE6D30978D6
S113093049060DD5FF2A08D300200AE0ADB24FF6D0
S1130940FF76B542F0D0002003E0002120F8121019
S1130950012070BC7047F0B44B730F23CB7200239B
S11309600B7300238B760023CB76D2B2531E0D2457
S1130970634300242500A4B2ADB24FF6FF76B5421E
S113098002D030F813505B1CDFF8006CA65D755480
S1130990DFF8F86BA65D7618ADB22F0A7770ADB2AA
S11309A0002D01D14FF6FF75641C0D2CE4D3ADB2BC
S11309B04FF6FF74A54203D030F81300002801D18C
S11309C052F040020A70F0BC70477CB50400160077
S11309D01D000B222000FFF78BFBADB2062D09DBB7
S11309E0ADB2E80310EB550031880D18B61C308801
S11309F00028F5D10720ADB2102195FBF1F202FBDE
S1130A00115212F13001C9B23A2900DBC91D00AA02
S1130A108154401EADB2102195FBF1F5ADB2002D0D
S1130A20E9D100A97E224254002100E0491C814200
S1130A3002D20A5D202AF9D10A00511C082803D2E7
S1130A4000ABC35C401C00E0202313550829F3D3FA
S1130A5073BD00210B22C9B2CB0113EB5101037802
S1130A605918401C521E002AF5D10800C0B2704724
S1130A702DE9F041050000212800FFF7B9FD04002D
S1130A80E4B2002C02D02000C0B226E0FF27B84612
S1130A9029692868FFF783FB0400E4B2002C1AD10B
S1130AA06E693078C0B2002801D1042413E0F17AD1
S1130AB011F03F01C0B2E52804D00A070FD5C9B22E
S1130AC00F290CD0FF2700212800FFF7E8FD0400C0
S1130AD0E4B2002CDCD02000C0B2BDE8F081C9B281
S1130AE00F291ED1E9690029EDD0410606D596F8F3
S1130AF00D8010F0BF000700E9882984C0B2FFB25E
S1130B00B8420CD1707B5FFA88F8804507D1310078
S1130B10E869FFF79FFE002801D07F1E00E0FF2751
S1130B20D1E7FFB2002F06D13000FFF792FF5FFA42
S1130B3088F88045CFD0FF274FF6FF702884A86936
S1130B40C07AC007BFD40B22A9693000FFF7E2FACC
S1130B500028B8D1BFE72DE9F04104000D00FF26BD
S1130B60FF275FF00408206900282ED0216920683F
S1130B70FFF715FB80465FFA88F8B8F1000F24D11F
S1130B8060690278D2B2002A02D15FF004081CE046
S1130B90C17A11F03F01D2B2E52A0BD0D2B22E2A8B
S1130BA008D0C9B2082901D1012300E00023DBB237
S1130BB0AB4215D0FF2600212000FFF770FD8046D0
S1130BC05FFA88F8B8F1000FCDD05FFA88F8B8F171
S1130BD0000F01D0002020614046C0B2BDE8F08182
S1130BE0C9B20F2919D1510605D5477B12F0BF02AE
S1130BF01600E1882184D2B2F6B2B2420BD1417B15
S1130C00FFB28F4207D10100E069FFF76EFE0028B2
S1130C1001D0761E00E0FF26CDE7F6B2002E04D107
S1130C20FFF717FFFFB2874202D04FF6FF70208410
S1130C30CBE72DE9F04184B00400A669E7690C22F2
S1130C40310000A8FFF754FA9DF80B00C0072CD51B
S1130C500020F0720020E0615FF0010801E018F16B
S1130C6001081FFA88F8B8F1640F0DDA43469BB205
S1130C703A0000A93000FFF7A8FE2000FFF7F8FEB5
S1130C800500EDB2002DEAD01FFA88F8B8F1640F20
S1130C9001D107207DE0EDB2042D02D02800C0B2BE
S1130CA077E09DF80B00F072E7619DF80B00800778
S1130CB012D55FF0000801E018F101081FFA88F866
S1130CC037F818000028F7D11FFA88F818F119002E
S1130CD00D2190FBF1F600E00126B6B231002000B0
S1130CE0FFF773FD0500EDB2002D32D1761E300002
S1130CF080B200282DD0E088811B89B22000FFF744
S1130D0077FC0500EDB2002D23D1A069FFF7A1FE09
S1130D10070021692068FFF742FA0500EDB2002DB3
S1130D2017D13B00DBB23200D2B26169E069FFF750
S1130D3012FE20680121017100212000FFF7AFFCA1
S1130D400500EDB2002D04D1761E300080B20028DB
S1130D50DFD1EDB2002D1AD121692068FFF71FFA07
S1130D600500EDB2002D12D1202200216069FFF7A9
S1130D70C9F90B22A1696069FFF7BAF9A069C07AC1
S1130D8010F01800616908732068012101712800BE
S1130D90C0B204B0BDE8F08138B50400E588208C09
S1130DA04FF6FF71884201D1290000E0218C89B2FD
S1130DB02000FFF71DFCC0B200281BD12169206868
S1130DC0FFF7EDF9C0B2002810D16169E5220A707D
S1130DD0216801220A71E188ADB2A94206D200213C
S1130DE02000FFF75CFCC0B20028E7D0C0B20428A2
S1130DF000D10220C0B232BD2DE9F14F8846002057
S1130E00D8F8009001E019F1010999F800002F28A1
S1130E10F9D099F800005C28F5D00098C669002440
S1130E20250002E026F815706D1C14F80970641C86
S1130E30BFB2202F05DBBFB22F2F02D0BFB25C2F71
S1130E4009D114EB0900C8F80000BFB2202F1FDA43
S1130E505FF004081EE0FF2D01D3062090E0FFB2EE
S1130E600121380080B201F0FBFC0700BFB2002F63
S1130E7001D1062084E0BFB2802FD3DABFB239009B
S1130E80DFF8F408FFF756F90028CBD0062077E006
S1130E905FF0000800E06D1E002D09D016EB450040
S1130EA030F8027CBFB2202FF5D0BFB22E2FF2D083
S1130EB0002D01D1062063E0002026F815000B2246
S1130EC0202100988069FFF71DF9002400E0641CCC
S1130ED036F814002028FAD036F814002E28F6D05C
S1130EE0002C03D058F0030800E06D1E002D05D03F
S1130EF016EB450030F8020C2E28F6D15FF00009FD
S1130F00CB465FF0080A01E058F0030836F8147085
S1130F10641CBFB2002F35D1009880690078E528A1
S1130F2003D10098806905210170BAF1080F01D13D
S1130F305FEA89095FFA89F919F00C000C2805D0D9
S1130F405FFA89F919F00300032801D158F0020867
S1130F505FEA88700FD45FFA89F919F00300012859
S1130F6001D158F010085FFA89F919F00C0004282F
S1130F7001D158F008080098806980F80B8000209F
S1130F80BDE8F28FBFB2202FBED0BFB22E2F01D149
S1130F90AC42B9D1D34501D2AC4213D1BAF10B0F53
S1130FA002D158F00308B7E7AC4201D058F0030867
S1130FB0A542B1D32C005FF0080B5FF00B0A5FEA87
S1130FC08909A3E7BFB2802F10DB0021380080B26B
S1130FD001F046FC0700BFB2002F05D0BFB2DFF816
S1130FE09C07381810F8807C58F00208BFB2002F14
S1130FF007D0BFB23900DFF88807FFF79BF8002855
S113100003D05F2758F003080FE0BFB2B7F14100E7
S11310101A2802D259F0020907E0BFB2B7F1610001
S11310201A2802D259F00109203F009880690BF870
S113103000701BF1010B69E7F8B50C0004F209011B
S11310400269002A48D04269137B00250EE0F6B2FB
S1131050052E00D1E5261F0705D5F6B2B6F14107E6
S11310601A2F00D220360E70491C6D1C082D03D295
S1131070AE5CF6B2202EEAD1157A202D15D02E259D
S11310800D70491C08250AE0DF0605D5F6B2B6F155
S113109041071A2F00D220360E70491C6D1C0B2DEF
S11310A003D2AE5CF6B2202EEED1D37A2372D37F74
S11310B0957F2D0455EA0363557F53EA0523157F75
S11310C02B432360537E157E55EA0323A380D37DEF
S11310D0927D52EA0322E28000220A70A16900296B
S11310E026D0E169002923D0A669002501690029D9
S11310F01CD0018C4FF6FF72914217D0C76901E0F2
S1131100A8556D1C3888BF1C010089B200290DD078
S1131110002180B201F0A4FB80B2002801D1002597
S113112004E0E169491E8D42EAD300250020A85558
S1131130F1BD13B50400019800782F2803D001985D
S113114000785C2802D10198401C01900020A06026
S11311500198007820280AD200212000FFF748FADD
S11311600021616120E02068FFF757FBA06001A91E
S11311702000FFF741FEC0B2002815D12000FFF780
S113118077FCA169C97AC0B2002806D0C0B204288D
S11311900AD1490700D4052006E0490704D461694F
S11311A0C87AC006DFD40520C0B216BD10B504004D
S11311B001230A0014F13401607801F068F9002871
S11311C001D003202DE094F8330294F8321251EA4E
S11311D0002080B24AF65521884201D0022020E046
S11311E094F86C0094F86B10090251EA004094F8EA
S11311F06A100843DFF8741C884201D1002010E013
S113120094F8880094F88710090251EA004094F891
S113121086100843DFF8541C884201D1002000E006
S1131220012010BDF8B5150002681378B3F130063B
S11312300A2E05D253783A2B02D1921C026000E0A8
S1131240002600200860002E01D00B209DE1DFF86D
S1131250200C50F82640002C01D10C2095E10C60A4
S1131260207800280DD0607801F008F9C10708D46F
S1131270EDB2002D03D0400701D50A2085E10020FE
S113128083E1002020706670607801F054F8C10793
S113129001D5032079E1EDB2002D03D0400701D53B
S11312A00A2072E1002529002000FFF77FFF0600D5
S11312B0F6B2012E1CD10020C0B2002800D0401E7E
S11312C0C0B214EB001000F2F210017900290FD023
S11312D0C17A827A120452EA0161427A51EA022105
S11312E0007A50EA010529002000FFF75FFF06009D
S11312F0F6B2032E01D1012047E1F6B2002E01D04F
S11313000D2042E194F8400094F83F1051EA002087
S113131080B2B0F5007F01D00D2036E194F84B0087
S113132094F84A1051EA002080B200280DD194F8B4
S11313305B0094F85A10090451EA006094F85910BB
S113134050EA012094F858100843E06194F84410DE
S1131350E170C9B2012904D0C9B2022901D00D201B
S113136013E1C9B2484394F84110A170C9B20029ED
S113137003D04A1EC9B2114201D00D2005E194F8F0
S1131380461094F8452052EA012121812189102236
S1131390B1FBF2F303FB1213002B01D00D20F4E098
S11313A094F8481094F8472052EA012292B2002A95
S11313B00DD194F8571094F85620120452EA0161A2
S11313C094F8552051EA022194F854200A4394F8E1
S11313D0431094F8423053EA012189B2002901D123
S11313E00D20D2E089B24318268913EB16139A42D2
S11313F001D20D20C9E0D21AA678B2FBF6F2002A77
S113140001D10D20C1E0012640F6F677BA4200D39F
S113141002264FF6F677BA4200D30326921CA26145
S1131420256289B2491961625919E162F6B2032E43
S113143016D12089002801D00D20A6E094F863007D
S113144094F86210090451EA006094F8611050EABB
S1131450012094F860100843A062A069800015E0A0
S11314602189002901D10D208FE0616A4018A06212
S1131470F6B2022E02D1A069400007E0A069032160
S11314804843217E11F0010111EB5000E16900F2A3
S1131490FF10B1EB502F01D20D2076E05FF0FF304A
S11314A020610020E060F6B2032E60D1002060715C
S11314B094F8650094F8641051EA002080B2401951
S11314C060610123626914F13401607800F0DFFF88
S11314D000284CD194F8330294F8321251EA0020D7
S11314E080B24AF65521884241D194F8370094F8E5
S11314F03610090451EA006094F8351050EA0120CE
S113150094F834100843DFF8381A88422FD194F83D
S11315101B0294F81A12090451EA006094F8191293
S113152050EA012094F818120843DFF8181A884288
S11315301DD194F8230294F82212090451EA0060A0
S113154094F8211250EA012094F820120843E06034
S113155094F81F0294F81E12090451EA006094F8EA
S11315601D1250EA012094F81C12084320612670D1
S1131570DFF8D4090088401CDFF8CC190880E0802B
S113158000202063002020710020F2BDDC7B0000DD
S113159080B500280BD00168002908D001680978BB
S11315A0002904D00168C9888288914201D00920A9
S11315B008E00068407800F061FFC00701D503200F
S11315C000E0002002BDC0B2002801D00B2012E0D0
S11315D0C0B2DFF89C2852F82020002A01D0002352
S11315E01370002901D000220A70C0B2DFF88028ED
S11315F042F82010002070472DE9F2438CB004001B
S11316001500002C01D10920B3E00020206015F062
S11316101F0515F0FE0200A90CA8FFF703FE060043
S1131620F6B2002E40F0A38009A80690DFF81C094A
S113163007900C9900A8FFF77CFD0600059FF6B201
S1131640002E02D1002F00D106261C20054258D0BE
S1131650F6B2002E0AD0F6B2042E03D100A8FFF78A
S1131660E8FA060055F00805059F08E0F87A11210C
S1131670084201D0072602E0680700D50826F6B222
S1131680002E4CD128074AD501F0D1F8804687F8BE
S11316900E80404680B2000AF8735FEA184038743E
S11316A05FEA186078740020F87200203877002010
S11316B078770020B8770020F87739000098FFF792
S11316C0ACF8814600213800FFF7B8F800980121F2
S11316D00171B9F1000F22D00098D0F8308049464A
S11316E00098FEF7F6FE0600F6B2002E17D1009819
S11316F0B9F10101C16041460098FEF750FD0600B2
S11317000DE0F6B2002E0AD1F87AC00601D50426FF
S113171005E0A80703D5F87AC00700D50726F6B276
S1131720002E07D1280701D555F020050098006B3D
S1131730E0612762F6B2002E19D1A5713900009834
S1131740FFF76BF82061F87FB97F090451EA006064
S1131750797F50EA0120397F0843E0600020A060CF
S11317600020A061009820600098C088A08030000C
S1131770C0B20DB0BDE8F0831C7C0000047500000D
S1131780587C00002DE9F047050016001F000C00EE
S1131790002038602800FFF7FBFEC0B2002801D00B
S11317A0C0B2E7E0A879000601D50220E2E0A879FA
S11317B0C00701D40720DDE0E868A968401AB042F8
S11317C029D2060027E0C5F81890A8684FF40071E4
S11317D0B0FBF1F202FB1102D2F50078464500D2CB
S11317E0B0464246A8684FF40071B0FBF1F303FB26
S11317F01103581910F124012000FEF779FC18EBAD
S11318000404A86818EB0000A860386818EB00000E
S11318103860B6EB0806002E00F0AB80A8684FF4E1
S11318200071B0FBF1F202FB1102002ACDD1A868CD
S1131830400A29688978491E11EA00085FFA88F885
S1131840B8F1000F1AD1A868002801D1286903E073
S113185069692868FEF734FD022805D2A87950F09A
S11318608000A871022085E010F1010F05D1A8794C
S113187050F08000A87101207CE0686169692868E3
S1131880FEF712FD8146B9F1000F05D1A87950F099
S11318908000A87102206DE05FFA88F818EB09094E
S11318A05FEA562ABAF1000F37D0286880785FFAC9
S11318B088F81AEB0801884205D2286880785FFA14
S11318C088F8B0EB080A5346DBB24A462100286880
S11318D0407800F0DCFD002805D0A87950F08000A5
S11318E0A871012046E0A879400611D5A869B0EB9B
S11318F0090050450CD24FF4007215F12401A86977
S1131900B0EB09004FF4007303FB0040FEF7F0FB5B
S11319104FF4007000FB0AF871E7A86948453FF4EA
S113192052AFA879400613D50123AA6915F1240101
S11319302868407800F0F8FD002805D0A87950F018
S11319408000A871012015E0A87910F0BF00A871EB
S113195001234A4615F124012868407800F097FDD8
S113196000283FF430AFA87950F08000A87101201E
S113197000E00020BDE8F0872DE9F04705001600DF
S11319801F000C00002038602800FFF701FEC0B2E1
S1131990002801D0C0B270E0A879000601D5022069
S11319A06BE0A879800701D4072066E0E868301866
S11319B0E96888422DD200262BE0C5F81890A86863
S11319C04FF40071B0FBF1F202FB1102D2F5007882
S11319D0464500D2B04642462100A8684FF4007341
S11319E0B0FBF3FC0CFB130C1CEB05002430FEF7DE
S11319F07FFBA87950F04000A87118EB0404A86894
S1131A0018EB0000A860386818EB00003860B6EBEB
S1131A100806002E26D0A8684FF40071B0FBF1F23E
S1131A2002FB1102002ACAD1A868400A29688978F1
S1131A30491E11EA00085FFA88F8B8F1000F30D1A6
S1131A40A868002808D12869002809D1002128683D
S1131A50FEF774FD286103E069692868FEF76EFDEE
S1131A6000280CD1E868A968884201D2A868E86017
S1131A70A87950F02000A8710020BDE8F087012863
S1131A8005D1A87950F08000A8710220F5E710F183
S1131A90010F05D1A87950F08000A8710120ECE76E
S1131AA06861A879400613D50123AA6915F12401B8
S1131AB02868407800F038FD002805D0A87950F057
S1131AC08000A8710120D8E7A87910F0BF00A871A0
S1131AD069692868FEF7E8FB8146B9F1000F05D172
S1131AE0A87950F08000A8710220C6E75FFA88F850
S1131AF018EB09095FEA562ABAF1000F38D02868B2
S1131B0080785FFA88F81AEB0801884205D22868C1
S1131B1080785FFA88F8B0EB080A5346DBB24A468D
S1131B2021002868407800F0FFFC002805D0A8793F
S1131B3050F08000A87101209FE7A869B0EB09006C
S1131B40504510D24FF40072A869B0EB09004FF46D
S1131B50007101FB004115F12400FEF7C9FAA879D0
S1131B6010F0BF00A8714FF4007000FB0AF844E7BE
S1131B70A86948453FF421AFA868E9688842BFF4E2
S1131B801CAF01234A4615F124012868407800F06F
S1131B907EFC00283FF411AFA87950F08000A871B2
S1131BA001206AE738B504002000FFF7F1FCC0B259
S1131BB000284AD1A179890647D5A07940060FD5D6
S1131BC00123A26914F124012068407800F0ACFCE0
S1131BD0002801D0012039E0A07910F0BF00A071E5
S1131BE0E1692068FEF7DBFAC0B200282DD1256A2E
S1131BF0E87A50F02000E872E0682877E06880B264
S1131C00000A6877E068000CA877E068000EE877BF
S1131C1021692800FEF712FE00F009FEA8750100F4
S1131C2089B2090AE975010C2976000E687600204C
S1131C30A8740020E874A07910F0DF00A071206877
S1131C40012101712068FEF7C5FAC0B232BD10B59A
S1131C5004002000FFF7A6FFC0B2002801D1002134
S1131C602160C0B210BD2DE9F04104000D00200038
S1131C70FFF78EFC0600F6B2002E02D03000C0B290
S1131C80CCE0A079000601D50220C7E0E068A842B4
S1131C9003D2A079800700D4E568A0680027A76074
S1131CA0002D7BD0216889784FF4007202FB01F883
S1131CB0002810D0411EB1FBF8F16A1EB2FBF8F205
S1131CC08A4208D3401EB8F101018843A060A0688D
S1131CD02D1A606919E02069002815D100212068B7
S1131CE0FEF72CFC012805D1A07950F08000A071EA
S1131CF0022093E010F1010F05D1A07950F080008B
S1131D00A07101208AE020616061002807D145E0CC
S1131D106061A16818EB0101A160B5EB0805A84555
S1131D2009D2A17989071ED501002068FEF706FCB7
S1131D3000281CD14546A1686918A1604FF40071C0
S1131D40B5FBF1F202FB1152002A27D001002068F2
S1131D50FEF7AAFA0700002F1ED1A07950F08000E8
S1131D60A07102205AE001002068FEF7A9FA10F1E0
S1131D70010F05D1A07950F08000A07101204DE041
S1131D80022803D3216889698842C1D3A07950F01D
S1131D908000A071022041E017EB5527A0684FF4A2
S1131DA00071B0FBF1F202FB1102002A2AD0A069F3
S1131DB0874227D0A079400613D50123A26914F1E4
S1131DC024012068407800F0AFFB002805D0A079FA
S1131DD050F08000A071012020E0A07910F0BF0035
S1131DE0A07101233A0014F124012068407800F026
S1131DF04EFB002805D0A07950F08000A07101208E
S1131E000CE0A761E068A168884205D2A068E060A0
S1131E10A07950F02000A0713000C0B2BDE8F0817C
S1131E2031B58CB00C00002203A90CA8FFF7FAF915
S1131E300500EDB2002D15D100A80990DFF80C01C2
S1131E400A900C9903A8FFF774F90500EDB2002D70
S1131E5008D10898002804D0210003A8FFF7ECF863
S1131E6000E006252800C0B20DB030BD4641540044
S1131E704016002071B595B0012200A915A8FFF7FE
S1131E80D1F90400E4B2002C56D109A806902F48D9
S1131E900790159900A8FFF74CF90400E4B2002C50
S1131EA04AD1059D002D01D1062403E0E87AC0073C
S1131EB000D5072429000098FEF7AFFC0600E4B221
S1131EC0002C21D1E87AC0061ED5022E01D20224AC
S1131ED01AE0242200A90CA8FEF70AF90E960221A2
S1131EE00CA8FEF785FB0400E4B2002C0CD1002101
S1131EF00CA8FEF730FE0400E4B2002C00D1072445
S1131F00E4B2042C00D10024E4B2002C14D100A8C3
S1131F10FEF742FF0400E4B2002C0DD1002E04D0E1
S1131F2031000098FEF7D5FA0400E4B2002C03D186
S1131F300098FEF74FF904002000C0B216B070BD3F
S1131F4052526141727241617C160020D01000200F
S1131F502DE9FC4104000F00904600252600FFE710
S1131F60781E854213DA00AB012201A94046FFF72F
S1131F7009FC009801280AD19DF80400C0B20D287C
S1131F80EED03070761C6D1CC0B20A28E8D1002057
S1131F903070002D00D100242000BDE8F68130B55A
S1131FA083B004000D00E4B20A2C03D129000D20F3
S1131FB0FFF7F5FF8DF80040012401AB220000A9D2
S1131FC02800FFF7D9FC0198A04201D1012001E0CB
S1131FD05FF0FF303EBD70B504000D00002601E047
S1131FE0641C761C2078002809D029002078FFF78B
S1131FF0D6FF10F1010FF3D15FF0FF3000E03000A5
S113200070BD10B450F8041B81B102681218001D91
S113201050F8043BDC0744BFA9F10104E31852F86B
S1132020044B43F8044B091FF9D1EBE710BC70478C
S113203010B582B001220121DFF8F80700F0A9FDF4
S113204020215FF0402000F0D4FD202220215FF009
S1132050402000F09EFD00240AE0FF21DFF8D807AD
S113206000F0FCFE00A9DFF8D00700F016FF641CA6
S11320700A2CF2D320215FF0402000F0E7FD13BDCD
S113208000B583B0DFF8B40701F0DDF8DFF8B0077E
S113209001F0D9F8DFF8AC0701F0D5F834215FF08E
S11320A0402000F0D3FD0121DFF8880700F0A1FDF6
S11320B00A23022234215FF0402000F0B7FC0A23F7
S11320C002220121DFF86C0700F0B0FC012201219B
S11320D0DFF8600700F05DFD01F032FA082101919C
S11320E0DFF864170091002300220100DFF848079D
S11320F000F019FEDFF8400700F08EFEFFF798FFAE
S113210007BD1CB5DFF8300700F097FE01F018FAA0
S11321104408DFF83807844201D3DFF8344701F07C
S11321200FFA082101910094002300220100DFF836
S1132130080700F0F8FDDFF8000700F06DFE13BD9E
S1132140DFF81007007850F00100DFF80817087076
S1132150704780B5C0B20100DFF8DC0600F07EFEF7
S113216000A9DFF8D40600F098FE0098C0B202BDC2
S113217010B50400FF20FFF7ECFF207010BD38B548
S113218001F031FB10F5FA75FF20FFF7E2FF0400C0
S1132190E4B2FF2C03D001F026FBA842F4D3E4B24E
S11321A0FF2C01D1012000E0002032BD80B50122C6
S11321B00121DFF8800600F0ECFCFF20FFF7C9FFE7
S11321C001BD80B500220121DFF8680600F0E1FCC2
S11321D0FF20FFF7BEFFFFF7D2FF002801D0012048
S11321E002E0FFF7E3FF002002BDF8B504000D0094
S11321F001F0F9FA10F16407FF20FFF7AAFF0600C7
S1132200F6B2FF2E03D101F0EEFAB842F4D3F6B2DF
S1132210FE2E01D0002011E02000FFF7A9FF641C6E
S11322202000FFF7A5FF641CAD1E002DF4D1FF2094
S1132230FFF78FFFFF20FFF78CFF0120F2BD38B5B9
S113224004000D00FFF79BFF002801D1002024E0CB
S11322502800C0B2FFF77DFFEDB2FD2D1CD04FF476
S113226000752078FFF775FF641C2078FFF771FF75
S1132270641CAD1E002DF4D1FF20FFF76AFFFF2080
S1132280FFF767FFFF20FFF764FFC0B210F01F00E5
S1132290052801D0002000E0012032BD38B504003B
S11322A00D0020060AD514F07F0400213720FFF723
S11322B0F5FFC0B2022801DBC0B23BE0FFF776FFB6
S11322C0FFF77FFF002801D1FF2033E054F04000E6
S11322D0C0B2FFF73EFF280EC0B2FFF73AFF280C4A
S11322E0C0B2FFF736FF280AC0B2FFF732FF28005A
S11322F0C0B2FFF72EFF0125E4B2002C00D19525D2
S1132300E4B2082C00D187252800C0B2FFF721FFD2
S1132310E4B20C2C02D1FF20FFF71BFF0A25FF209B
S1132320FFF717FF010604D56D1E2900C9B2002965
S1132330F5D1C0B232BD70B582B0C0B2002801D0B0
S113234001209AE0DFF80C050078800703D5DFF858
S11323500405007891E0FFF793FE00220121DFF8E5
S1132360D40400F016FC002500210020FFF796FF9E
S1132370012869D101F037FA10F57A764FF4D57156
S11323800820FFF78BFF01283CD1002406E0FF2042
S1132390FFF7DFFEE4B200A96054641CE4B2042C2D
S11323A0F5DB9DF8020001284ED19DF80300AA2810
S11323B04AD101F018FAB04206D25FF08041A92058
S11323C0FFF76CFF0028F4D101F00DFAB0423BD2C4
S11323D000213A20FFF762FF002835D1002406E0EF
S11323E0FF20FFF7B6FEE4B200A96054641CE4B217
S11323F0042CF5DB9DF80000400601D50C2500E017
S1132400042521E00021A920FFF748FF022802DA71
S11324100225A92401E00125012401F0E4F9B042D8
S113242006D200212000C0B2FFF738FF0028F4D103
S113243001F0D9F9B04206D24FF400711020FFF731
S11324402DFF002800D00025DFF80C04EDB2056054
S1132450FFF7ACFEEDB2002D0AD0DFF8F8030078E8
S113246010F0FE00DFF8EC130870FFF74AFE01E0FD
S1132470FFF766FEDFF8DC03007876BDC0B2002803
S113248001D0012002E0DFF8CC030078704738B5B2
S11324900C0011001D00C0B2002802D1EDB2002DC5
S11324A001D104203FE0DFF8AC030078C00701D578
S11324B0032038E0DFF8A0030078000702D44FF4CB
S11324C000704143EDB2012D0DD11120FFF7E6FE5E
S11324D000281FD14FF400712000FFF786FE00286A
S11324E018D0002516E01220FFF7D8FE002811D1DD
S11324F04FF400712000FFF778FE002806D014F591
S113250000746D1E2800C0B20028F1D100210C20F7
S1132510FFF7C4FEFFF74AFEEDB2002D01D0012003
S113252000E00020C0B232BD70B50C0015001E00E2
S1132530C0B2002802D1F6B2002E01D1042050E02E
S1132540C4480078C00701D503204AE0C148007898
S1132550400701D5022044E0BF480078000702D4B8
S11325604FF400704543F6B2012E0DD12900182016
S1132570FFF794FE00282BD1FE212000FFF75FFE19
S1132580002825D0002623E0B348007810F0060F79
S113259004D0F6B231009720FFF780FE29001920FD
S11325A0FFF77CFE002813D1FC212000FFF747FE33
S11325B0002806D014F50074761E3000C0B200283E
S11325C0F2D1FD210020FFF73AFE002800D10126B8
S11325D0FFF7ECFDF6B2002E01D0012000E0002050
S11325E0C0B270BD30B585B014002200C0B200285E
S11325F001D0042019E197480078C00701D50320D1
S113260013E10125C9B2002913D0012917D00329E8
S11326105ED00A2900F0BB800B2900F0BD800C2994
S113262000F0C8800D2900F0D3800E2900F0E3806B
S1132630F6E0FFF7C6FD002800D00025F1E00021F8
S11326400920FFF72BFE002841D1102100A8FFF735
S1132650CCFD00283BD09DF80000C0B28009C0B278
S113266001280FD19DF809009DF8081010EB0120F6
S11326709DF8071011F03F0110EB0140401C80024F
S1132680206023E09DF8050010F00F009DF80A106B
S1132690C9B210EBD1109DF8091011F0030110EB31
S11326A04100851C9DF80800C0B28009C0B29DF8A5
S11326B0071010EB81009DF8061011F0030110EBD8
S11326C08120401CB5F10901884020600025A8E064
S11326D061480078400720D500218D20FFF7DEFDFA
S11326E0002853D1FF20FFF734FD102100A8FFF785
S11326F07CFD00284AD0302503E0FF20FFF729FDA8
S11327006D1EEDB2002DF8D110209DF80A10C9B24B
S1132710090988402060002538E000210920FFF7DE
S1132720BDFD002832D1102100A8FFF75EFD00286E
S11327302CD049480078800713D59DF80A0010F082
S11327403F009DF80B10C9B2C909C9B211EB400092
S1132750401C9DF80D10C9B28909491E88402060AB
S113276013E09DF80A00C0F38400C0B2401C9DF839
S11327700B1011F003019DF80B20D2B25209D2B212
S113278012EBC101491C48432060002549E032484E
S113279000681070002544E000210920FFF77EFD49
S11327A0002806D110212000FFF71FFD002800D0CB
S11327B0002536E000210A20FFF770FD002806D12D
S11327C010212000FFF711FD002800D0002528E08B
S11327D000213A20FFF762FD00280BD1002505E017
S11327E0FF20FFF7B6FCEDB228556D1CEDB2042DA9
S11327F0F6DB002515E01848007840070FD50021C6
S11328008D20FFF74BFD002809D1FF20FFF7A1FC25
S113281040212000FFF7E9FC002800D0002500E05B
S11328200425FFF7C3FC2800C0B205B030BD0B4837
S1132830704700000070004000800040100000104D
S11328400100002008000020801A060021BCBE0000
S113285020BCBE0001000020441600200000AA4253
S113286080B2802801DA01001EE000290CD080B279
S1132870FF2801DD002106E080B2194911EB400078
S1132880B0F5807001880FE0002100E0491C89B296
S1132890802906DA89B2124A32F8112080B29042B5
S11328A0F4D111F18000C1B2080080B27047002158
S11328B000E0491C0B4A32F81120002A05D0094ACD
S11328C032F8112080B29042F3D1064A32F8112036
S11328D0002A03D0044830F81100FFE780B27047A3
S11328E044730000846F000064710000B0F1402F55
S11328F05BD0DFF83813884257D0DFF834138842AE
S113290053D0DFF8301388424FD0DFF82C138842BD
S11329104BD0DFF82813884247D0DFF824138842CD
S113292043D0DFF8201388423FD0DFF81C138842DD
S11329303BD0DFF85013884237D0DFF84C1388427D
S113294033D0DFF8481388422FD0DFF8441388428D
S11329502BD0DFF84013884227D0DFF83C1388429D
S113296023D0DFF8381388421FD0DFF834138842AD
S11329701BD0DFF86813884217D0DFF8641388424D
S113298013D0DFF8601388420FD0DFF85C1388425D
S11329900BD0DFF85813884207D0DFF8541388426D
S11329A003D0DFF85013884201D1012000E0002059
S11329B0C0B2704770B504000D0016002000FFF788
S11329C095FF002805D14FF49071DFF82C0300F037
S11329D019FF002E09D0012E07D0022E05D04FF486
S11329E09171DFF8140300F00DFFF00705D514F51D
S11329F080600068EDB2284304E014F5806000684C
S1132A00EDB2A84314F580610860B00705D514F54C
S1132A1084600068EDB2284304E014F58460006823
S1132A20EDB2A84314F58461086070BDF8B50400E4
S1132A300D0017001E002000FFF758FF002805D1E5
S1132A4040F2FF11DFF8B00200F0DCFE012F0BD0E2
S1132A50022F09D0042F07D00C2F05D040F20321F8
S1132A60DFF8940200F0CEFE082E0DD00A2E0BD013
S1132A700C2E09D0092E07D0002E05D04FF4027178
S1132A80DFF8740200F0BEFEF80705D514F5A06067
S1132A900068EDB2284304E014F5A0600068EDB2CC
S1132AA0A84314F5A0610860B80704D5D4F8040558
S1132AB0EDB2284303E0D4F80405EDB2A843C4F80A
S1132AC00405780705D514F5A1600068EDB2284324
S1132AD004E014F5A1600068EDB2A84314F5A16107
S1132AE00860380705D514F5A3600068EDB22843E3
S1132AF004E014F5A3600068EDB2A84314F5A361E3
S1132B000860F00704D5D4F80C05EDB2284303E0BF
S1132B10D4F80C05EDB2A843C4F80C05B00705D5EC
S1132B2014F5A2600068EDB2284304E014F5A26035
S1132B300068EDB2A84314F5A2610860700704D5DB
S1132B40D4F81405EDB2284303E0D4F81405EDB22B
S1132B50A843C4F81405300704D5D4F81C05EDB215
S1132B60284303E0D4F81C05EDB2A843C4F81C05BF
S1132B70002E05D114F5A5600068EDB2284304E0E9
S1132B8014F5A5600068EDB2A84314F5A5610860CA
S1132B90F1BD70B504000D0016002000FFF7A6FE7D
S1132BA0002805D140F28531DFF84C0100F02AFEFF
S1132BB0EDB2F6B244F8256070BD38B504000D00DE
S1132BC02000FFF793FE002805D140F25241DFF8C0
S1132BD0280100F017FE02222900C9B22000FFF7E5
S1132BE0E9FE082304222900C9B22000FFF71EFFD2
S1132BF031BD38B504000D002000FFF777FE002832
S1132C0005D140F2F141DFF8F00000F0FBFD0823AC
S1132C1001222900C9B22000FFF708FF0122290080
S1132C20C9B22000FFF7C6FE31BD00000080054098
S1132C3000500040009005400060004000A00540A6
S1132C400070004000B005400040024038B5040068
S1132C500D002000FFF74AFE002804D140F29661DF
S1132C60254800F0CFFD02222900C9B22000FFF759
S1132C70A1FE082301222900C9B22000FFF7D6FED5
S1132C8031BD000000C005400050024000D00540A6
S1132C900060024000E005400070024000F0054082
S1132CA000D0034038B504000D002000FFF71EFEDD
S1132CB0002804D140F2EA610F4800F0A3FD02228B
S1132CC02900C9B22000FFF775FE0823012229005C
S1132CD0C9B22000FFF7AAFE31BD00000000064083
S1132CE00010064000200640003006400040064028
S1132CF00050064000600640D0770000DFF8C011A5
S1132D0088420BD0DFF8BC11884207D0DFF8B81135
S1132D10884203D0DFF8B411884201D1012000E0D9
S1132D200020C0B270472DE9F84304000F001500DD
S1132D3099462000FFF7E2FF002804D1CC21DFF8F8
S1132D40900100F05FFD002D0ED0022D0CD0012D5E
S1132D500AD0032D08D0102D06D0202D04D0D22166
S1132D60DFF86C0100F04EFDB9F1000F0AD0B9F1A3
S1132D70010F07D0B9F1020F04D0D521DFF85001BB
S1132D8000F040FDDDF82080B9F1000F02D1780891
S1132D9040450BD2B9F1000F04D00C20B7FBF0F082
S1132DA0404503D2D7214A4800F02CFDB7FBF8F088
S1132DB0B0F57E4F03D9D821454800F023FD099E84
S1132DC0301F0D2803D3D921414800F01BFDB9F170
S1132DD0020F01D1082000E00020B9F1000F01D159
S1132DE0002100E0042108436060B7FBF8F00021F3
S1132DF0891CB0FBF1F2521EFF2AF9D8216115F0AB
S1132E000300800115F0300550EA02202843711EAA
S1132E1008432060BDE8F18310B504002000FFF7EB
S1132E206DFF002804D14FF48571294800F0EAFCB5
S1132E30606850F00200606010BD10B5040020000E
S1132E40FFF75CFF002804D140F22311204800F072
S1132E50D9FC606830F00200606010BD38B5040031
S1132E600D002000FFF74AFF002804D140F223217F
S1132E70174800F0C7FC7FF00100216811F00F0132
S1132E808840054204D040F22521114800F0BAFCE4
S1132E90E0688007FCD5A56031BD38B504000D009D
S1132EA02000FFF72BFF002804D140F27F210848BF
S1132EB000F0A8FCE0684007FCD5A068286031BD9C
S1132EC0008000400090004000A0004000B000409E
S1132ED02C780000DFF8DC13884200F04A81DFF828
S1132EE0D813884200F04581DFF8D013884200F0FF
S1132EF04081DFF8CC13884200F03B81DFF8C41333
S1132F00884200F03681DFF8C013884200F0318136
S1132F10DFF8B813884200F02C81DFF8B41388423C
S1132F2000F02781DFF8AC13884200F02281DFF83B
S1132F30A813884200F01D81DFF8A013884200F036
S1132F401881DFF89C13884200F01381DFF8941392
S1132F50884200F00E81DFF89013884200F0098166
S1132F60DFF88813884200F00481DFF88413884274
S1132F7000F0FF80DFF87C13884200F0FA80DFF86D
S1132F807813884200F0F580DFF87013884200F06F
S1132F90F080DFF86C13884200F0EB80DFF86413F4
S1132FA0884200F0E680DFF86013884200F0E18098
S1132FB0DFF85813884200F0DC80DFF854138842AD
S1132FC000F0D780DFF84C13884200F0D280DFF89D
S1132FD04813884200F0CD80DFF84013884200F0A7
S1132FE0C880DFF83C13884200F0C380DFF8341354
S1132FF0884200F0BE80402800F0BB80B0F1102F62
S113300000F0B780DFF82013884200F0B280DFF8C8
S11330101C13884200F0AD80DFF81413884200F0DE
S1133020A880DFF81013884200F0A380DFF8801432
S1133030884200F09E80DFF87C14884200F099807A
S1133040DFF87414884200F09480DFF8701488422A
S113305000F08F80DFF86814884200F08A80DFF87F
S11330606414884200F08580DFF85C14884200F024
S11330708080B0F1101F7CD0DFF85014884278D0E3
S1133080DFF84C14884274D0DFF84814884270D0BA
S1133090DFF8441488426CD0DFF84014884268D0CA
S11330A0DFF83C14884264D0DFF83814884260D0DA
S11330B0DFF8341488425CD0DFF83014884258D0EA
S11330C0DFF82C14884254D0DFF82814884250D0FA
S11330D0DFF8241488424CD0DFF82014884248D00A
S11330E0DFF81C14884244D0DFF81814884240D01A
S11330F0DFF8141488423CD0DFF81014884238D02A
S1133100DFF80C14884234D0DFF80814884230D039
S1133110DFF8041488422CD0DFF80014884228D049
S1133120DFF8FC13884224D0B0F1202F21D0DFF83F
S1133130F41388421DD008281BD0DFF8EC13884212
S113314017D0DFF8E813884213D0DFF8E41388427D
S11331500FD0DFF8E01388420BD0DFF8DC1388428D
S113316007D0DFF8D813884203D0DFF8D01588429F
S113317001D1012000E00020C0B2704710B582B038
S113318004002000FFF7A6FE002805D140F23131EB
S1133190DFF8A40500F036FB14F0704010F1805FF6
S11331A023D1C4F30720DFF898150818E1B2890089
S11331B051EA401050F08440012101600020009049
S11331C002E00098401C009000981028F9D3C4F342
S11331D00720DFF86C150818E1B2890051EA4010A5
S11331E050F08440002101602CE0200FDFF85815D6
S11331F051F820000068A1B2220C12F01F02914085
S11332000843210FDFF8402552F821100860002000
S1133210009002E00098401C009000981028F9D318
S1133220200FDFF8241551F820000068A1B2220C09
S113323012F01F0291408843210FDFF80C2552F849
S11332402110086013BD10B504002000FFF742FEF2
S1133250002805D140F29631DFF8DC0400F0D2FA00
S113326014F0704010F1805F0DD1C4F30720DFF833
S1133270D4140818E1B2890051EA401050F0844097
S11332800121016011E0200FDFF8C01451F8200083
S11332900068A1B2220C12F01F0291400843210FD2
S11332A0DFF8A82452F82110086010BD0138FDD1C0
S11332B07047704701001000020010000001100068
S11332C00002100000041000000110100002101091
S11332D000041010005800F000401010005010209E
S11332E0005400F00100002002000020040000202F
S11332F008000020100000202000002040000020D2
S11333008000002000010020090800F00A0800F0F5
S11333100B0800F00C0800F00D0800F00E0800F097
S11333200F0800F0100800F000400010022000F028
S1133330032000F0042000F070B50400DFF81C0442
S1133340006810F0E04F08D0DFF810040068DFF8E0
S113335010140840B0F1805F02D1002C00F1A78066
S1133360DFF8EC030568DFF8FC03066855F4006534
S113337035F4800556F40066DFF8D4030560DFF801
S1133380E4030660A80701D5A00708D515F00100DD
S113339014F0010191F00101C0B208421ED074F092
S11333A003000540DFF8A8030560002E07D516F0DA
S11333B07000302809D016F07000702805D0002E57
S11333C008D415F03000302804D14FF48050FFF7B2
S11333D06DFF03E05FF40020FFF768FF35F4FE653E
S11333E014F4FE600543DFF880030640DFF87C0335
S11333F02040064314F0080056EAC006DFF85003E4
S11334000560DFF8600306601020FFF74FFF35F416
S1133410405514F44050054336F4005614F400505B
S11334200643DFF8300340210160002E06D5DFF8A3
S113343034030660DFF81803056005E0DFF81003C5
S11334400560DFF820030660DFF824030540DFF899
S113345024032040054336F0FC5614F0FC50064388
S1133460600008D555F4800536F48006DFF80803BB
S11334702040064301E036F0804620050ED44FF488
S1133480004000E0401E002804D0DFF8CC12096898
S11334904906F7D535F4006536F40066DFF8B00266
S11334A00560DFF8C00206601020FFF7FFFE70BD64
S11334B0052000F00010101000011020004800F05A
S11334C080000030005000F010000030014000F097
S11334D00001001000020010100000102000001075
S11334E0021C00F0031C00F020000030010010104A
S11334F0020010100400101008001010040400F062
S1133500050400F001000010020000100400001087
S1133510031800F0041800F0051800F0061800F075
S1133520071800F00100102000101000005C00F0EB
S1133530015C00F0025C00F0035C00F0045C00F04D
S113354030B4DFF80C020168DFF818020268002AC0
S113355002D512F0700001E011F0300000280DD007
S113356010283AD020286FD0302800F0A48060289A
S113357000F0A480702800F0A480A5E0C1F38410BA
S1133580DFF8F83153F82000DFF8F431134013F179
S1133590004F05D0002A00F1AA800B0500F1A78096
S11335A0DFF8E0311B68DFF8B441246814F0E04F21
S11335B009D0DFF8A8412468DFF8A4512C40B4F105
S11335C0805F40F08380C3F34814A41C604313F06D
S11335D01F04A41CB0FBF4F081E0DFF88001006854
S11335E010F0E04F08D0DFF874010068DFF87031A4
S11335F01840B0F1805F02D1DFF88C0123E0DFF8DE
S11336005C010068DFF858311840DFF880319842D7
S113361005D1DFF84801006880B202280ED0DFF837
S11336203C010068DFF838311840DFF86431984213
S113363007D1DFF828010068000402D1DFF8540143
S113364001E0DFF854019FE7DFF81001006810F093
S1133650E04F08D0DFF804010068DFF804311840B7
S1133660B0F1805F02D1DFF8340123E0DFF8EC0031
S11336700068DFF8EC301840DFF81031984205D1CB
S1133680DFF8D800006880B202280ED0DFF8CC0042
S11336900068DFF8CC301840DFF8F430984207D1E6
S11336A0DFF8B8000068000402D1DFF8F40001E09C
S11336B0DFF8F00068E747F2305065E75FF4800018
S11336C062E74FF400405FE7002032E0C3F34814A0
S11336D0604313F01F04641C6400B0FBF4F05C044A
S11336E000D540081B0400D5800851F480014B022A
S11336F01FD5002A18D5530010D5DFF884301340A5
S113370013F1004F03D0002A08D4090506D4400061
S1133710C2F38651491CB0FBF1F00AE0C2F3C55173
S1133720491CB0FBF1F004E0C1F3C351491CB0FBE8
S1133730F1F030BC70470000B0760000055C00F08A
S113374000E50F4000E60F40347C0000407C0000A0
S113375060E00F4058E00F4050E00F4000E00F40A1
S11337600000FF7070E00F408FFFFF7F300000808B
S1133770FCFF3FF80300C0070000404084750000D0
S11337800008008064E00F40C0E1E4000000011084
S113379000000310001BB7000024F4007038390047
S11337A0C0C62D0000093D0080B500F00EF8114898
S11337B04CF24F3101601048002101600F4805218F
S11337C001600F480021016001BD0C480021016027
S11337D070470A480068C00304D509480068401CC3
S11337E007490860704780B5FFF7F3FF0448006895
S11337F002BD000014E000E018E000E010E000E08A
S11338005016002080B500F002F8FCE770477047BE
S1133810C2788A18DFF81832DA70827889B20B0A13
S11338209A18DFF80C329A70DFF804224378537048
S1133830DFF8FC2100781070DFF8F401807889B299
S11338400A0AD2B2904212D2DFF8E4014078401C56
S1133850DFF8DC215070DFF8D8014078002806D169
S1133860DFF8CC010078401CDFF8C4211070DFF8C9
S1133870C001C07889B2C9B2884217DADFF8B00152
S11338808078401C6A4988706948807800280DD186
S113389067484078401C664948706548407800286D
S11338A004D163480078401C61490870704710B423
S11338B092B25218531E0AE00A784C7814EB022292
S11338C0101880B292B2904200D2401C891C9942D6
S11338D0F2D3994207D109780A02101880B292B241
S11338E0904200D2401C80B210BC704780B51422B4
S11338F050490020FFF7DBFF80B2002802D14FF6C9
S1133900FF7002E080B201F05FF880B202BD10B532
S11339104949097C484A527C12EB0121B1F1140453
S1133920C0B200190822454980B2FFF7C0FF220047
S113393092B2434980B2FFF7BAFF80B2002802D1A5
S11339404FF6FF7002E080B201F03EF880B210BD85
S113395080B50620FFF7DBFF02BD3A480021017065
S11339600AE0384800783849002221F81020354808
S11339700078401C33490870324800780028F0D0A1
S11339803048002101700CE02E48007868212F4A4D
S113399001FB0020002141762A480078401C294977
S11339A00870284800780028EED029484FF4806138
S11339B001807047234900220A7004E021490978F4
S11339C0491C204A11701F49097800290CD11D494E
S11339D009781D4A32F811100029EFD119490978E4
S11339E0194A22F81100FFE7704780B5010089B237
S11339F0DFF8DC0D00680830FFF70AFFDFF8D00DB0
S1133A0000680B4909780172DFF8C40D00680849A1
S1133A1049784172DFF8B80D0068054989788172E8
S1133A20DFF8AC0D00680249C978C17201BD00001D
S1133A307416002012000020040000201E00002044
S1133A40260000208F160020821600205414002027
S1133A508616002010B5DFF8781D0C68DFF8C41D49
S1133A60DFF8C42D1160DFF8C42D1160C0B2032843
S1133A7018D1607E10F00F0003280AD1208A002894
S1133A8007D1DFF8AC0D0821017001F03CF800F01B
S1133A9064BEDFF8A00D00210180DFF8940D002141
S1133AA0017010BDC0B2022840F0CB80DFF8880D51
S1133AB0C078401CDFF8801DC870C0B200281AD13D
S1133AC0DFF8740D8078401CDFF86C1D8870C0B27C
S1133AD0002810D1DFF8600D4078401CDFF8581D35
S1133AE04870C0B2002806D1DFF84C0D0078401CA5
S1133AF0DFF8441D0870DFF83C0D00210180DFF879
S1133B003C0D00210180607E072802D0607E0528DC
S1133B1008D1A07E401CA076A07E782801D1002088
S1133B206076B6E7607E0028FBD0208A00287AD031
S1133B30A07E411EA176C0B20028F2D1E07E082802
S1133B4008D0607E022802D0607E012810D1E07E79
S1133B5005280DD100206076DFF8D40C8021017097
S1133B6000F0D1FFDFF8A40D142180F82F108DE1AF
S1133B70E07E052801DB042000E0E07E032111FA49
S1133B8000F0A076E07E401CE076607E10F00F002E
S1133B90C0B201280AD0022835D0032839D004281D
S1133BA03FD006283DD008283BD0BAE7DFF85C0DAB
S1133BB0102180F82F10DFF8540D90F82F0050F0EA
S1133BC00200DFF8481D81F82F00DFF8400D0221C4
S1133BD080F83610DFF8340D042180F83710DFF850
S1133BE02C0D062180F83810DFF8200D0A2180F80A
S1133BF03910DFF8400C2C210180DFF8100D602112
S1133C0080F82E104BE1DFF8040D002180F82F100E
S1133C10D1E7DFF81C0C0421017000F074FF00F000
S1133C20DEBD00F041BD607E10F00F0003287FF47C
S1133C3078AFDFF8FC0B0821017000F064FF00F09E
S1133C408CBDDFF8C80C807B45287FF422AFDFF8F9
S1133C50E40B0088DFF8B41C097CDFF8B02C527C3C
S1133C6012EB0121884216DBDFF8A00C007CDFF8A0
S1133C709C1C497C11EB0020DFF8B81B0880DFF89E
S1133C808C0C007D3F21084204D1DFF8800C407D7C
S1133C90002801D0FDE6FCE6DFF8240D0088DFF8FB
S1133CA0241D0988884207D1DFF8140D4088DFF805
S1133CB0141D4988884210D0DFF8500CC08BDFF8FF
S1133CC0001D0988884207D1DFF8400C008CDFF81A
S1133CD0F01C4988884200D0DBE6FFF707FE4FF668
S1133CE0FF7188427FF4D5AEDFF8200CC07D062832
S1133CF008D1FFF72DFE4FF6FF71884244D1DFF85B
S1133D00F84C43E0DFF8040CC07D01287FF4C1AE19
S1133D10DFF8F80B90F8220008287FF4BAAEDFF839
S1133D20EC0B002180F82210DFF8E00B808C4FF6BA
S1133D30F771884207DBDFF8D40B808C0930DFF899
S1133D40CC1B888406E0DFF8C40B808C0830DFF8D5
S1133D50BC1B8884DFF8B40BDFF8B01B498BC1832C
S1133D60DFF8A80BDFF8A41B898B0184DFF89C0B18
S1133D70DFF84C1C09884183DFF8900BDFF8401C06
S1133D804988818300F016BE83E66834DFF8680C46
S1133D90A042C0F0DB80607E0028F6D0DFF86C0B18
S1133DA0808CA1888842F0D1DFF8600B408CE188D8
S1133DB08842EAD1DFF8540B408B21888842E4D151
S1133DC0DFF8480B808B61888842DED1DFF8000A77
S1133DD00460DFF85C0A00210170DFF8300B90F812
S1133DE02F00400700F1BC82DFF8200B90F82E0072
S1133DF0C0B200098000DFF8041C0870DFF8340A40
S1133E000088DFF8F81B0978401A1438DFF8241A00
S1133E100880607E10F00F00022808D1DFF8EC0A59
S1133E2090F82F0010F03F00122800F0A382DFF872
S1133E30040A0088002807D1DFF8D00A90F82F0080
S1133E400321084200F09682DFF8C00A90F82600A9
S1133E50217A884215D1DFF8B40A90F82700617AF4
S1133E6088420ED1DFF8A40A90F82800A17A88428B
S1133E7007D1DFF8980A90F82900E17A884200F027
S1133E807982DFF8880A102180F82F10DFF8A4095E
S1133E9028210180DFF8740A502180F82E10DFF801
S1133EA06C0A217A80F82A10DFF8600A617A80F8B7
S1133EB02B10DFF8580AA17A80F82C10DFF84C0A8E
S1133EC0E17A80F82D10DFF8440A217B80F826106F
S1133ED0DFF8380A617B80F82710DFF8300AA17B0D
S1133EE080F82810DFF8240AE17B80F82910DFF835
S1133EF01C0A0621C175DFF8140AA1884184DFF881
S1133F000C0AE1888184DFF8040ADFF8B41A09880E
S1133F104183DFF8F809DFF8A81A49888183DFF8BC
S1133F20EC092188C183DFF8E40961880184607E9B
S1133F30C00640F1F9840020DFF8D01981F831007F
S1133F40DFF8C81981F8300000F0F6BCDFF8BC09CE
S1133F5090F82F0010F03F00022806D0DFF8AC09DB
S1133F6090F82F00400729D593E5DFF8A009808C4D
S1133F70DFF88C1A0880DFF8840A0021017006E05B
S1133F80DFF8780A0078401CDFF8701A0870DFF850
S1133F906C0A00780028E1D1DFF8640A0088DFF8B1
S1133FA05C1A0978DFF85C2A32F811108842E7D1EC
S1133FB00024DFF8480A00210170E6E0DFF84C092C
S1133FC0142180F82F10DFF86C0828210180DFF815
S1133FD03C09502180F82E10DFF8300990F82900B0
S1133FE0DFF8181A0870DFF82409DFF8201991F8AF
S1133FF02D1080F82910DFF81409DFF8001A097869
S113400080F82D10DFF8040990F82800DFF8EC1987
S11340100870DFF8F808DFF8F41891F82C1080F82D
S11340202810DFF8E808DFF8D419097880F82C1094
S1134030DFF8D80890F82700DFF8C0190870DFF817
S1134040CC08DFF8C81891F82B1080F82710DFF897
S1134050BC08DFF8A819097880F82B10DFF8AC0841
S113406090F82600DFF894190870DFF8A008DFF84C
S11340709C1891F82A1080F82610DFF89008DFF8D1
S11340807C19097880F82A10DFF8800890F82D0050
S1134090401CDFF8781881F82D00C0B2002820D128
S11340A0DFF8680890F82C00401CDFF8601881F8ED
S11340B02C00C0B2002814D1DFF8500890F82B006F
S11340C0401CDFF8481881F82B00C0B2002808D142
S11340D0DFF8380890F82A00401CDFF8301881F81F
S11340E02A00DFF82808408CDFF814190880DFF86C
S11340F01C08DFF81818898C4184DFF81008DFF8F1
S1134100001909888184DFF80408DFF80018498B56
S1134110C183DFF8F807DFF8F417898B0184DFF82F
S1134120EC07DFF89C1809884183DFF8E007DFF823
S113413090184988818300F0FFBBDFF8C00800783D
S11341406821DFF8B42801FB0020407E072815D140
S1134150002C0BD0A07EDFF8A41809786822DFF8C1
S1134160983802FB0131897E884207D2DFF88C0837
S113417000786821DFF8802801FB0024DFF87C0840
S11341800078401CDFF874180870DFF870080078B5
S1134190002812D1DFF8640800786821DFF8582875
S11341A001FB0020407E0028C7D1DFF850080078CA
S11341B06821DFF8442801FB0024002C3FF469AC9B
S11341C0DFF80C0604600320A07620760020A0759A
S11341D00420E0750020E076DFF83007808CA080B2
S11341E0DFF82807408CE080DFF82007408B208030
S11341F0DFF81807808B608001206076DFF83806CE
S113420000782073DFF8300640786073DFF8280602
S11342108078A073DFF82006C078E0730120208244
S1134220DFF8E80690F82900E072DFF8E00690F87D
S11342302800A072DFF8D40690F827006072DFF837
S1134240CC0690F8260020720120FFF7CEFBDFF8A1
S1134250BC0690F82E0010F0F0005128FFF6A6AC32
S1134260DFF898070021017006E0DFF89007007876
S1134270401CDFF888170870DFF880070078DFF843
S11342808C1691F82E10C9B20909C9B2491FB0EBB6
S1134290810FBFF68BACDFF864070078DFF86C168B
S11342A0401890F83600DFF860170870DFF85807F8
S11342B0007800283FF47AACDFF84C070078012836
S11342C0D3D0DFF84407007802282ED1DFF82C077A
S11342D00078DFF83816401890F83700042824D105
S11342E0DFF818070078DFF82416401890F8380033
S11342F0DFF808170978DFF81426891891F83910BF
S113430051EA0020DFF8F8160880DFF8F406008888
S113431040F20B61884202DB40F20A6002E0DFF8FF
S1134320E00600886082A08240E4DFF8D0060078CE
S1134330DFF8D815401890F8370000283FF436AC61
S1134340DFF8B8060078DFF8B4160978DFF8BC2582
S1134350891891F837100818DFF8A01608708BE751
S113436000206076DFF8C8042021017000F0CBFB48
S1134370FFF78FBBDFF8940590F82F00C00664D5D3
S1134380208A002861D0218A14F10C00FFF740FA3A
S1134390DFF8780590F82A00DFF87016097888426B
S11343A053D1DFF8680590F82B00DFF860164978E0
S11343B088424AD1DFF8540590F82C00DFF84C16F7
S11343C08978884241D1DFF8440590F82D00DFF860
S11343D03C16C978884238D1DFF83006007820735B
S11343E0DFF8280640786073DFF820068078A07331
S11343F0DFF81806C078E073E07E00281DD194F938
S1134400180094F91A10401AA17DC9B2B0EBD1007A
S1134410A17D4118A17540B2002801D540B24042A7
S1134420E17DC9B2B0EB9100E17D4018E075A07D5B
S1134430C0B2E17D11EBD0002076DFF8F403012156
S11344400170207EA07600202082607E10F00F0094
S1134450C0B2012813D0C0F06582032800F0FA80AE
S113446035D3052800F02F82C0F0F881072800F02A
S11344704F82C0F04F82082800F0E48152E2DFF856
S1134480B0030078C00720D503206076DFF8A003CE
S11344904021017000202082DFF898030088002862
S11344A00CD0DFF88C03007850F00200DFF88013A2
S11344B00870DFF880030088FFF797FADFF87C03C1
S11344C00021018000F01FFB47E1FFF7E2BADFF8AB
S11344D060030078C00740F1B380DFF8300490F83F
S11344E02F0010F03F00122840F0AA80DFF81C04CF
S11344F090F82E0010F0F000512829DBDFF8FC04BE
S11345000021017006E0DFF8F4040078401CDFF8B5
S1134510EC140870DFF8E4040078DFF8F01391F885
S11345202E10C9B20909C9B2491FB0EB810F0FDAC5
S1134530DFF8C8040078DFF8D413401890F8360088
S1134540DFF8C4140870DFF8C0040078002826D10E
S113455003206076DFF8B40390F826002072DFF8B9
S1134560AC0390F827006072DFF8A00390F82800ED
S1134570A072DFF8980390F82900E0720120FFF799
S113458034FAAB484221017000202082A94800215E
S11345900180AA480021018000F0B5FADDE0DFF8CF
S11345A0680400780128AED0DFF85C0400780228A3
S11345B02ED1DFF848040078DFF85013401890F843
S11345C03700042824D1DFF834040078DFF83C13E2
S11345D0401890F83800DFF824140978DFF82C2309
S11345E0891891F8391051EA0020DFF81414088072
S11345F0DFF80C04008840F20B61884202DB40F2D1
S11346000A6002E0DFF8F80300886082A0829FE776
S1134610DFF8E8030078BD49401890F83700002817
S113462096D0DFF8D8030078DFF8D0130978B74ABA
S1134630891891F837100818DFF8C013087069E773
S11346407B482021017000F05EFA61480068002177
S1134650417683E4AD4890F82F00C0072AD5607EE8
S1134660C00627D4208A00287FF413AA7148008842
S1134670401C80B2FFF7B9F96D48007850F0100083
S11346806B4908706B480088002805D0684800789A
S113469050F002006649087000F035FA01202082CB
S11346A0082060760020E0769848112180F82F10C9
S11346B0FFF7ECBB954890F82F00800619D5934876
S11346C090F83400914991F8351051EA0020564988
S11346D00968401854490860564800888B4991F885
S11346E034108A4A92F8352052EA0121401A51497D
S11346F008805048008800280CD0607EC00609D489
S11347004B48007850F00200494908704948008835
S1134710FFF76BF97D4890F830007C4991F831102F
S113472011EB0020B6490880A08AB549098888425F
S113473003D3B3480088002802D1A08AB049088076
S1134740AF48008860823A4800780321084277D055
S11347503A480021018000F0D6F9354800788006F7
S11347600AD536480021018000206076674814216C
S113477080F82F10FFF78ABB2D480078C0060ED5AD
S11347802E48002101800120208204206076002030
S1134790E0765E48112180F82F10FFF777BB274899
S11347A00088002819D022480078C00701D50020CD
S11347B02082208A00280DD1608A204909888842F5
S11347C002D2608A1D4908801C480088208204E0C7
S11347D06C160020208A194908800020E0761248CF
S11347E01249096801601548008800280CD0208A05
S11347F0002809D0208A28300E490880434818210F
S113480080F82F10FFF746BB09480078800717D5BA
S11348100848282101803D48102180F82F10FFF717
S113482039BB00BF3A00002064160020681600203F
S11348308E1600207E1600207016002080160020A0
S1134840FFF727B972480078C00706D500206076C4
S11348506F481021017000F056F963E06D4800883C
S1134860002803D06B480088FFF7BFF8274890F86A
S11348702F00C00716D566480078C00706D5072064
S113488060760020A0760020208201E00620607679
S11348900120FFF7AAF85E481021017000F033F9F7
S11348A0FFF7EFBA5A480078C00705D505206076AF
S11348B000202082FFF7EDB85648008800287FF4D6
S11348C0E0AAFFF7E6B853480088002803D051480F
S11348D00088FFF78AF80D4890F82F00C0070DD51F
S11348E0072060760020A0760120FFF77EF8484874
S11348F01021017000F007F9FFF7C3BA454800889A
S113490000287FF4BEAAFFF7C4B800BF040000204B
S1134910FFF7B7BA3E480078C00703D50720607692
S11349200020A076FFF7B5B83B48062180F8301088
S113493039480A2180F831103748402181753648BA
S11349403449098889B2090A01743348314909880C
S113495041740020304981F835002F4981F8340032
S11349602D4800214186FEF7F3FFC0432A494886BB
S113497029484521817328480021C1730020264914
S113498048752549087525480088401C2349088036
S113499021482249098889B2090A81741E481F499D
S11349A00988C1741C4800210183FEF79FFFC0439E
S11349B019490883164800210170FFF772B80000F6
S11349C058160020807C000080B2010A51EA0020C1
S11349D080B2704780B501290CDB114A118011495E
S11349E00968884206D00E490A8801000D4800680B
S11349F000F038F901BD0000541400208F16002087
S1134A0088160020821600209016002074160020BC
S1134A108E1600207E16002004000020841600203C
S1134A20801600206816002080B500F033F9FEF7E8
S1134A30DAFE10F5FA7080490860FEF7D4FE00F53E
S1134A401C5010307D490860FEF787FF4FF6A960BF
S1134A50ADF8000043F61370ADF802007848BDF8D5
S1134A60001001807648BDF8021041804FF6FF70B7
S1134A70ADF800000020ADF802007248BDF8001047
S1134A8001807048BDF8021041804FF6A960ADF86E
S1134A90000040F21310ADF802006B48BDF800109E
S1134AA001806948BDF8021041804EF60300FEF70C
S1134AB081FF00F0F7F801BD38B5644A126812F1BD
S1134AC01C0422686260002205E092B2131992B2BB
S1134AD0155C1D72521C0B00DBB292B29BB29A425F
S1134AE0F3D3C9B2081DA4F84800B4F84810201D37
S1134AF0FFF770FF2068401C206031BD80B500F0D6
S1134B0032F8002002BD10B55048006810F11C04B2
S1134B104F480078400605D5012020600020A4F805
S1134B2048001FE04A480078C00702D50020A4F8D6
S1134B30480047480078400708D5B4F848000028E2
S1134B4004D0B4F84810201DFFF744FF4048007813
S1134B50800707D50020A4F848003E480068001DDF
S1134B6000F080F910BD10B500F026F900282DD012
S1134B70394908804FF40060FFF726FF37498989D7
S1134B8080B281420ED10120FEF764FF32480088D2
S1134B9000281BD000F0B7FC00F023F92E480021B8
S1134BA0018013E040F60600FFF70EFF2B498989C8
S1134BB080B281420AD100F040FC274800880028D6
S1134BC004D000F00EF9244800210180FEF70BFE0A
S1134BD01949096888421ED31748006810F5FA700D
S1134BE015490860002414E068201D4900FB0410E6
S1134BF0164908600220FEF72DFF17480088002898
S1134C0006D000F080FC00F0ECF81348002101808D
S1134C10641C002CE8D0FEF7E6FD084909688842C8
S1134C2008D30648006800F51C501030034908609A
S1134C3000F038FB10BD0000481600204C16002080
S1134C4058160020601600205C1600206C16002008
S1134C508E160020641600207E160020040000201A
S1134C605414002010B50400200000F025FD20009D
S1134C7010BD50F8041B61B150F8042BD30744BF96
S1134C80A9F101039A18002342F8043B091FFAD141
S1134C90EFE7704780B55748FEF7D5FA5548FEF759
S1134CA06DFA01BD30B585B05348FEF7CCFA0C213E
S1134CB05248FDF782FF7F21514800F08FFE00210A
S1134CC04F4800F0A3FE040021004D4800F0B0FE60
S1134CD0FEF736FC01004A4800F02AFD1621484838
S1134CE000F03AFD464800F08BFD0121444800F0F5
S1134CF0B5FE0400FEF777FD00F59855883560078A
S1134D0008D401213E4800F0A9FE0400FEF76BFD23
S1134D10A842F4D308208DF8000000208DF801008B
S1134D2027208DF8020069208DF803005B208DF8A0
S1134D30040045208DF8050002A903A800F03FFFF8
S1134D40039810F1010F19D0029810F1010F15D03A
S1134D5003988DF800000398000A8DF80100039869
S1134D60000C8DF8020002988DF803000298000AE6
S1134D708DF804000298000C8DF8050000A9204865
S1134D8000F014FD1F489DF8001001701D489DF8A7
S1134D90011041701B489DF80210817019489DF85C
S1134DA00310C17017489DF80410017115489DF84F
S1134DB00510417105B030BD10B50021104800F058
S1134DC025FE040021000E4800F032FEE00706D55F
S1134DD040F242620C490A4800F074FD00E00020F1
S1134DE010BD80B5094802880749054800F0D3FD85
S1134DF001BD00000050102020000020005002409F
S1134E000080044034160020040000207E16002098
S1134E10DFF8700400210170DFF868040021816468
S1134E20DFF86004002180F84310DFF85804002103
S1134E30A0F84410DFF84C0400218170DFF844042A
S1134E40002141707047DFF83C040078002801D14C
S1134E50002000E001207047DFF82804002180F8DA
S1134E604310704780B50178FF291ED100F091F8F6
S1134E70DFF8100490F84300012802D1102000F05C
S1134E807EF8DFF80004B0F9440001280CDBDFF8F9
S1134E90F403012180F84310DFF8E803B0F944106B
S1134EA0DFF8E40300F053F801BDDFF8D813097804
S1134EB001294BD10178C92932D0CC293FD0CF293F
S1134EC03AD0D0292FD0D12933D0D2292ED0F329CA
S1134ED017D0F4290FD0F5290AD0F6290ED0FA29D3
S1134EE012D0FC2913D0FD2914D0FE2915D029E0B5
S1134EF000F0DAF8BCE700F0F9F8B9E700F0C9F817
S1134F00B6E700F018F9B3E700F0ABF8B0E700F04B
S1134F10A2F8ADE700F087F8AAE700F075F8A7E774
S1134F2000F03DF9A4E700F05CF9A1E700F01AF9FC
S1134F309EE700F087F99BE700F098F998E700F006
S1134F40ABF995E7202000F01AF891E7ACE780B5BB
S1134F5089B200F0A4FE01BD10B4002302E004787D
S1134F60E318401C0C00611E002CF8D1DBB2136066
S1134F70012010BC7047C348002141707047C149EB
S1134F80FE22CA70BF490871BE480221A0F844102D
S1134F90704710B5040000F0E0FE002803D1102093
S1134FA0FFF7EDFF2FE0FFF7E6FFB64801210170A0
S1134FB0B448FF21C170B34800210171B1480079A0
S1134FC050F01000AF490871AE4800214171AD485E
S1134FD0AC494979417100F07AFEAA49887100F020
S1134FE08BFEA849C87100F087FE80B2000AA5496B
S1134FF00872A44801214172A24801218172A1488A
S11350000821A0F8441010BD10B504009D480021EB
S11350100170FFF7B0FF9B48FF21C170994801213F
S1135020A0F8441010BD9749FF22CA709549002288
S11350300A719449934A52784A71924900228A71BA
S113504090490022CA718F4900220A728D490622B2
S1135050A1F84420704710B504000020FFF78FFF2B
S113506010BD8849FF22CA708649884A8A648549E6
S113507000220A71834900224A71824900228A71FE
S113508080490722C1F807207E490822A1F844205C
S113509070477C49FF22CA707A494068886479481D
S11350A00121A0F84410704710B5040000F00FFE71
S11350B0401E6178884203DA2220FFF760FF14E083
S11350C0627892B26F48816C714801F023FA6D489E
S11350D0FF21C1706B48806C617808186949886445
S11350E06078401C6749A1F8440010BD10B5040065
S11350F000F0EDFD401E6178884203DA2220FFF7BC
S11351003EFF17E05F4861688164627892B25D484F
S1135110816C5F4801F0FEF95A48FF21C17059487B
S1135120806C61780818574988646078401C554938
S1135130A1F8440010BD80B55249FF22CA70554AF7
S113514041685048806CFFF707FF4E4908714D488D
S1135150002141714B48002181714A480821A0F87F
S1135160441001BD10B504004648FF21C1704548F4
S11351700021017143480021417100F0A8FD41491B
S1135180887140480021C1713E48002101723D48A8
S1135190002141723B480721A0F8441010BD10B50E
S11351A0040000F094FD621C80B2411E3548806CFE
S11351B001F0C5F9002803D13120FFF7E0FE0FE02C
S11351C03048FF21C17000F082FD2E49896C80B205
S11351D0401E40182B4988642A480121A0F8441035
S11351E010BD10B5040000F072FD801E6178884285
S11351F003DA2220FFF7C3FE23E02248FF21C17017
S113520020480121A0F844106078002807D101F05B
S1135210A6F9002802D13120FFF7B1FE11E0A21C4B
S113522061781848806C01F08AF9002803D1312094
S1135230FFF7A5FE05E01348806C61780818114952
S1135240886410BD80B541680E48806C01F07BF91C
S1135250002803D13120FFF792FE06E00948FF2120
S1135260C17008480121A0F8441001BD10B5040024
S113527001F036F90348FF21C17002480121A0F86A
S1135280441010BD1C1500201F150020787C000060
S1135290201500202315002080B53120FFF76FFE74
S11352A001BD000080B5DFF8C8030078401CDFF8BA
S11352B0C0130870DFF8B003002101701EE0DFF8AE
S11352C0A80300780C21DFF8A42301FB0020018847
S11352D04288114300290AD0DFF894130978827AAE
S11352E0891A782903DB0422002101F042F9DFF84E
S11352F078030078401CDFF870130870DFF8680347
S113530000780828DBDB01BD38B50C00DFF8581342
S113531000220A7006E0DFF850130978491CDFF810
S113532048231170DFF84013097808291FDADFF8E1
S1135330381309780C22DFF8343302FB013529884D
S11353400029E8D069880029E5D001882A8891429B
S1135350E1D141886A889142DDD106222100281DCD
S1135360FFF780FCDFF808030078A87264E0DFF838
S1135370F81200220A7006E0DFF8EC120978491CE2
S1135380DFF8E4221170DFF8E012097808290DDA59
S1135390DFF8D41209780C22DFF8D03202FB013591
S11353A029880029E8D169880029E5D1AE4909781E
S11353B0082934D1AF4900220A70AF4900220A708B
S11353C0A94900220A701CE0A74909780C22A74BBE
S11353D002FB0135A7490978A54A1278AB7AD21A9B
S11353E0914209DAA2490978AA7A891AA14A117064
S11353F0A1499D4A12780A709B490978491C9A4A26
S11354001170994909780829DEDB97499A4A12787C
S11354100A70954909780C22944B02FB0135042249
S113542001002800FFF71EFC06222100281DFFF7BB
S113543019FC8F480078A87231BD80B58F48008868
S11354402A2803D28D48002101805BE08B4800218B
S113545001808B48808AB0F5807F03D0B0F5007F4F
S113546040D04FE08648C08C86490988884238D1AC
S11354708348008D83494988884232D182498348D0
S1135480FFF742FF7E484FF40071818206227E4975
S11354907F48FFF7E7FB06227E497B48FFF7E2FBE4
S11354A006227C497C48FFF7DDFB062278497448D4
S11354B0FFF7D8FB72487249898BC18470487049E0
S11354C0C98B01856E486F49098881836C486D4991
S11354D04988C1836A484FF4C161818167482A21A0
S11354E001800FE06648C08C66490988884209D16A
S11354F06348008D63494988884203D162496348FF
S1135500FFF702FF01BD80B55D49C98B634A12886C
S113551091420BD15A49098C604A5288914205D173
S113552006225F495648FFF79DFB8EE05449C98B1C
S11355305C4A12881140534A12885A4B1B881A40FD
S113554091420BD14E49098C564A528811404D4A1A
S11355505288544B5B881A40914208D05249534AAE
S113556012880A805049514A52884A8007E04449C7
S1135570C98B4D4A11804C49414A128C4A803A49A0
S113558000220A7004E038490978491C364A11702F
S11355903549097808290FDA334800780C21334A51
S11355A001FB00204049098802889142EBD13E4921
S11355B0498842889142E6D12B49097808293FD18C
S11355C00622FF212E4800F0D4FF06220021304895
S11355D000F0CFFF06222F492F48FFF743FB062296
S11355E02C492948FFF73EFB25482F490988C184E7
S11355F023482D4949880185214822490988818306
S11356001F4820494988C1831D484FF48071818215
S11356101B484FF48071C181194808210182184840
S11356200621817416480421C17415484FF4C161E0
S113563081811F481F49016010482A21018011E01F
S11356400622011D0E48FFF70DFB062211491248E0
S1135650FFF708FB0A4808218181084800880E30BA
S11356600649088001BD000091160020BC140020EA
S11356709316002094160020921600207E16002017
S113568004000020581600201A00002020000020EA
S113569024000020341600200A000020847C00002E
S11356A0707C000060160020781600205C16002034
S11356B0641600203A00002062B38B0708D0521E03
S11356C011F8013B00F8013B00F024808B07F6D170
S11356D0830740F0208000BF103A07D330B4B1E80C
S11356E03810103AA0E83810F9D230BC530724BF60
S11356F0B1E80810A0E8081044BF51F8043B40F892
S1135700043BD20724BF31F8022B20F8022B44BFFC
S11357100B7803707047083A07D3B1E80810083AC9
S113572040F8043B40F804CBF7D25307E4E7000009
S113573038B504000D00DFF85C03844204D05D2119
S1135740DFF85403FEF75EF86808DFF85013B0FB87
S1135750F1F0C0B2606231BD38B504000D00DFF86D
S11357603403844204D0A621DFF82C03FEF74AF860
S1135770DFF82C03054204D0AA21DFF81C03FEF74E
S113578041F8E06830F01600E9B20843E060A06830
S113579030F00E00C5F307210843A060E06B400819
S11357A04000C5F307410843E06331BD70B582B0E2
S11357B004000D0000AEDFF8DC02844205D040F2A4
S11357C01311DFF8D402FEF71DF8002D05D14FF4B4
S11357D08A71DFF8C402FEF715F82878307068780B
S11357E07070A878B070E878F0700098606100205C
S11357F0009028793070687970700098A06173BD4A
S113580010B50400DFF88C02844205D040F269111F
S1135810DFF88402FDF7F6FFA06850F01000A060E6
S1135820A06850F00100A060E06850F00100E06062
S1135830A06850F01000A06010BDF0B40024056909
S1135840ABB22E0C6654641C2D0E6554641C9D1F53
S1135850AA4201DA160004E09E1F02E005696550C1
S1135860241D351FA542F9DAB44220DA0569F71E72
S1135870BC4209D16554641C2E0A6654641C2D0C68
S11358806554641C641C12E0B71EBC4206D1655406
S1135890641C2D0A6554641CA41C08E0761EB442E2
S11358A005D16554641CE41C01E00569241D991E9E
S11358B08C42FADB9B1F9A4201DA584200E018003E
S11358C0F0BC704770B504000D001600DFF8C40189
S11358D0844204D040F28F216F48FDF793FF002DDE
S11358E004D14FF424716C48FDF78CFF012E04DAC7
S11358F040F291216848FDF785FF606B10F03F0F7F
S113590001D1002004E0320029002000FFF795FFB8
S113591070BD30B403001000002240F2FF74A042B6
S113592001DB404235E0B0F10E04555C54EA054415
S1135930521C555C54EA0564521C1C6102E0545824
S11359401C61121D041F9442F9DA82421FD0C41E46
S1135950A2420BD1545C521C555C54EA0524521CDF
S1135960515C54EA0144521C1C6110E0841EA242A2
S113597007D1545C521C515C54EA0124521C1C6132
S113598005E0441EA24202D1545C521C1C61012158
S1135990996330BC704770B504000D0016003D4893
S11359A0844204D040F29E313B48FDF72BFF002D8A
S11359B004D140F29F313848FDF724FF012E04DA68
S11359C04FF468713448FDF71DFFA06BC007FCD489
S11359D0320029002000FFF79CFF70BD38B5040099
S11359E00D002C48844204D040F247412A48FDF778
S11359F009FFE809C001002804D040F24A412648C2
S1135A00FDF700FF6068A843606031BD38B504004D
S1135A100D002048844204D040F26A411E48FDF73C
S1135A20F1FE2068EDB2002D01D06168084032BD5E
S1135A3038B504000D001748844204D040F29F4159
S1135A401548FDF7DFFEE809C001002804D040F244
S1135A50A2411148FDF7D6FE256031BD38B50400DA
S1135A600D000C48844204D040F212510A48FDF75C
S1135A70C9FE206AC007FCD4EDB2E80010F0F800BB
S1135A8050F001002062206AC007FCD4206B80B271
S1135A9032BD000000800440F0750000A0252600FF
S1135AA0E9F1FEFF10B50400A00504D09C21DFF845
S1135AB06001FDF7A7FEDFF85C0140F601210160FB
S1135AC0DFF854010460DFF85401DFF85411016079
S1135AD0DFF8480100688007FAD4DFF8480100685D
S1135AE040F60121084202D05FF0FF3000E00020C0
S1135AF010BD70B504000D00160015F0030F04D09E
S1135B00DF21DFF80C01FDF77DFE16F0030F04D052
S1135B10E021DFF8FC00FDF775FEDFF8F80042F243
S1135B2001610160DFF800010068C00739D5002E6B
S1135B3039D0E809C001DFF8E010086008E015F08A
S1135B407C00DFF8E81022680A50241D2D1D361F42
S1135B5015F07C0F04D1DFF8D8000068002801D1CB
S1135B60002EECD1DFF8CC00DFF8CC100160DFF8B8
S1135B70C4000068C007FAD4D9E7DFF89C000560C8
S1135B80DFF8B80021680160DFF89000DFF8A810A2
S1135B900160DFF888000068C007FAD4241D2D1DB9
S1135BA0361F002EE9D1DFF87C00006842F2016163
S1135BB0084202D05FF0FF3000E0002070BD38B52D
S1135BC005000C00002D04D14FF421711048FDF79D
S1135BD019FE002C04D140F285210D48FDF712FE78
S1135BE01748006810F0E04F06D0154800681549C2
S1135BF00840B0F1805F02D15FF0FF3006E0124848
S1135C0000682860114800682060002032BD000050
S1135C105076000014D00F4000D00F4008D00F4041
S1135C20020042A40CD00F40A0E10F4000D10F406D
S1135C3030D00F4020D00F40010042A404D00F40C8
S1135C4000E00F400000FF70E0E10F40E4E10F408E
S1135C5080B5FFF7DDF800F097FC324800210170B1
S1135C60FEF7E2FE2F480321017001BD80B52E48E6
S1135C7000F0C4FC012805D12A48002101702A48FB
S1135C80FFF7F0F82848FEF739FF012805D1254829
S1135C90032101702448FFF7E5F801BD704738B5CA
S1135CA004000D001F480078002804D12900C9B25F
S1135CB0200000F077FC1B480078032804D1290059
S1135CC0C9B22000FEF7F8FEFFF7C6F831BD15484B
S1135CD00078002805D0022807D004D3032806D072
S1135CE007E0402006E0002004E0002002E040201D
S1135CF000E0402080B270470A480078002805D0B0
S1135D00022807D004D3032806D007E0402006E089
S1135D10002004E0002002E0402000E0402080B2A7
S1135D207047000000000020AC15002080B5FFF78C
S1135D308AF802BD80B5DFF8780600210170DFF82B
S1135D4074160020FBF73FFCC0B2002804D0772172
S1135D50DFF86406FDF756FD01BDDFF85406007850
S1135D60002801D1012000E00020704780B5FFF732
S1135D70DDFF012801D1002011E0DFF834060078AE
S1135D80002801D000200AE000F0AEFC012805D173
S1135D90DFF81C0601210170012000E0002002BD93
S1135DA010B50024DFF808060078002800F0FF8111
S1135DB0DFF8FC050078012834D100F0AFFCDFF8EF
S1135DC0FC0500F0E0FCDFF8F80500F0DCFC00F076
S1135DD0A3FC01220100DFF8EC05FBF70DFC002811
S1135DE007D0DFF8E40500F0CEFC012000F0C1FC90
S1135DF0DDE1DFF8D80500F0C6FCDFF8D40500F0DB
S1135E00C2FCDFF8D00500F0BEFCDFF8CC050021B1
S1135E100160DFF8C40500214160DFF89405022128
S1135E200170C4E1DFF888050078022840F0F780AB
S1135E30DFF890254FF48071DFF8A005FCF788F8AF
S1135E40DFF8701591F83A12C1F3C01111F0010195
S1135E5001290FDBDFF8700500F095FC022000F04B
S1135E6088FCDFF86005FBF7F2FEDFF8440500214B
S1135E7001709CE100281BD00022DFF86415DFF8D4
S1135E805C0500F0D5F9040024B214F1010F0FD120
S1135E90DFF8340500F077FC032000F06AFCDFF83B
S1135EA02405FBF7D4FEDFF80805002101707EE12C
S1135EB024B2012C28DBDFF82005406800280BD130
S1135EC0DFF81805D0F88001DFF80C150860DFF85A
S1135ED0080524B2446017E0DFF80005D0F880011B
S1135EE0DFF8F4140968884206D2DFF8F004D0F829
S1135EF08001DFF8E4140860DFF8DC04406824B2B1
S1135F002018DFF8D4144860DFF8A804D0F83C0265
S1135F10DFF8A014D1F84012884201D1012000E03A
S1135F2000200128C0F243810021DFF89804FBF728
S1135F309AFE00280FD0DFF8900400F024FC04201F
S1135F4000F017FCDFF87C04FBF781FEDFF8600447
S1135F50002101702BE1DFF8740400F014FCDFF879
S1135F60840400F010FCDFF88014DFF86C0440684F
S1135F7000F074FADFF8700400F005FCDFF86C043C
S1135F8000F001FCDFF86014DFF84C040068000E38
S1135F90C0B200F052FADFF85814DFF83C0400688D
S1135FA0000CC0B200F049FADFF84814DFF8280406
S1135FB00068000AC0B200F040FADFF83C14DFF8D1
S1135FC018040068C0B200F038FADFF81C0400F0CE
S1135FD0DAFB77A000F0D7FBDFF8FC034168DFF8B9
S1135FE0F803006800F0AFFA00280FD1DFF8D803F7
S1135FF000F0C9FB052000F0BCFBDFF8C803FBF789
S113600026FEDFF8AC0300210170D0E0DFF8BC030A
S113601000F0B9FBDFF8980303210170C7E0DFF853
S113602090030078032840F0C280DFF898234FF4EF
S11360308071DFF8A803FBF78BFFDFF8781391F882
S11360403A12C1F3C01111F0010101290EDBDFF88E
S1136050AC0300F098FB022000F08BFBDFF8640334
S1136060FBF7F5FDD24800210170A0E000281AD00A
S1136070DFF88C23DFF86813DFF8600300F0D8F84A
S1136080040024B214F1010F0DD1DFF8780300F0FD
S11360907AFB032000F06DFBCA48FBF7D8FDC44827
S11360A00021017083E024B2012C4CDBD64800F0BF
S11360B06AFBCD4924B2200000F0D0F9CA4800F0B0
S11360C062FBD24800F05FFBC749C448D0F88001A6
S11360D0000EC0B200F0B1F9C549C048D0F8800143
S11360E0000CC0B200F0A9F9C249BC48D0F8800144
S11360F0000AC0B200F0A1F9BF49B848D0F8800145
S1136100C0B200F09AF9B84800F03DFB28A000F0B6
S11361103AFBBB4A24B22100B048D0F8800100F019
S11361200EFA00280CD1A84800F02DFB062000F040
S113613020FBA448FBF78BFD9D480021017036E04D
S1136140A24800F020FB9B48D0F83C029949D1F8C2
S11361504012884201D1012000E00020012826DB02
S1136160AB4800F010FB00F0FAF900280CD1964877
S113617000F009FB072000F0FCFA9248FBF767FDEA
S11361808B480021017012E0904800F0FCFAA1480D
S113619000F0F9FA8B48FBF75AFD9F4800F0F3FA38
S11361A083480021017000F0CAFA00F099F910BD8B
S11361B02E2E2E0010B50400207800F00FFB53287B
S11361C004D1607800F00EFB002801D103200FE019
S11361D06078312801D100200AE06078322801D1AA
S11361E0012005E06078332801D1022000E003207B
S11361F010BD70B504000026A41C200000F047F96F
S11362000500AE19A41C200000F041F986196D1E8A
S1136210A41CADB2022DF6DAF6B2F643200000F06B
S113622036F9F6B2864201D0002000E0012070BDAC
S11362302DE9F04105000E0014005FF00008002E67
S113624001D0002D04D140F231215B48FDF7DAFA88
S11362502800FFF7AFFF0700FFB2032F01D1002092
S1136260A3E02800FFF7C5FF002802D15FF0FF304C
S11362709BE0FFB2002F03D0022F5AD028D392E024
S1136280AD1C280000F003F90700AD1C280000F045
S1136290FEF800023060AD1CD6F80080280000F043
S11362A0F6F810EB08003060AD1CB7F10308002CC1
S11362B00DD0002606E0280000F0E9F8B6B230550B
S11362C0AD1C761CB6B20FFA88F84645F3DB6AE0DB
S11362D0AD1C280000F0DBF80700AD1C280000F01E
S11362E0D6F800043060AD1CD6F80080280000F019
S11362F0CEF818EB00203060AD1CD6F800802800E2
S113630000F0C5F810EB08003060AD1CB7F10408CC
S1136310002C0DD0002606E0280000F0B8F8B6B234
S11363203055AD1C761CB6B20FFA88F84645F3DB3F
S113633039E0AD1C280000F0AAF80700AD1C2800C5
S113634000F0A5F800063060AD1CD6F800802800E7
S113635000F09DF818EB00403060AD1CD6F80080CA
S1136360280000F094F818EB00203060AD1CD6F83B
S11363700080280000F08BF810EB08003060AD1CA2
S1136380B7F10508002C0DD0002606E0280000F027
S11363907EF8B6B23055AD1C761CB6B20FFA88F84A
S11363A04645F3DBFFE7404600B2BDE8F08100005C
S11363B08B1600204806002074790000507A0000F3
S11363C0007A00007C080020607C0000687C0000EB
S11363D0747A0000A47900002C160020D01200204A
S11363E050140020287C0000EC150020047B0000E1
S11363F0EE150020F0150020F2150020987A000018
S1136400D0130020BC7A0000EC7B0000587B000015
S1136410207B0000707B0000D479000080B501006F
S113642011F00F003030C9B20A2901DBC01D02E0AF
S1136430C0B200F0D3F9C0B202BD38B504000D00FB
S1136440E4B22009FFF7EAFF287014F00F00FFF709
S1136450E5FF68700020A870280032BD0200491CC6
S11364600A23B2FBF3F2002AF9D100220A700200D7
S1136470491E0A20B2FBF0F300FB132030300870F1
S11364800A20B2FBF0F2002AF2D10800704770B57E
S113649004000025002609E03038C0B20A2800DBD9
S11364A0C01FEDB2C0B210EB0515761CF6B2022E79
S11364B00FDAF6B2305D00F091F9C0B2B0F13001FC
S11364C0172904D2C0B2B0F13A010729E4D200205E
S11364D001E02800C0B270BD80B500F08BF901BDA9
S11364E010B500F034F800280FD0FFF7D7FBFDF704
S11364F06CF900F030F8054908400549086000F0DF
S11365002AF8446800F078F9A04710BD80FFFF1F07
S113651008ED00E070B504000D00160005E02878D1
S113652020706D1C641CFDF772F93000461E80B2A9
S11365300028F4D170BD80B500F060F901BD80B5CC
S113654000F067F902BD80B500F08DF902BD80B599
S113655000F0E6F902BD80B500F025FA02BD80B571
S113656000F09BF9002801D1002001E000F000FABE
S113657002BD10B5040010000A000100200000F064
S113658061FB200010BD000080B54F48FCF75BFEA6
S1136590FCF7D6FF60234FF4614201004B4800F042
S11365A0AAFB01BD70B504000D00EDB2412D03DB63
S11365B05B214748FDF726F92800C0B200F071F8C6
S11365C0C0B2012803D05F214148FDF71BF9002622
S11365D00DE0FDF71CF9B6B2305D00F062F8C0B210
S11365E0012803D068213A48FDF70CF9761C2800ED
S11365F0C0B2B6B280B28642EBD370BD10B504000F
S113660034480078002813D1334800F03DF80128BD
S113661038D131480078002834D0FDF7E4F82F4908
S113662008602F48002101702A480121017029E0E7
S11366302B48007828494018401C00F025F8012810
S113664016D127480078401C254908702448007852
S113665021490978884215D12148027892B221490A
S11366602000FFF757FF1B480021017001200AE0BA
S1136670FDF7B9F8194909686431814202D2154815
S113668000210170002010BD10B504000F4800F077
S1136690F0FB10F1010F02D02070012000E0002077
S11366A010BD80B50100C9B2084800F0F7FB00280E
S11366B003D1002007E0FDF7AAF8044800F0C3FB6B
S11366C00028F8D0012002BD0100001000C00040E5
S11366D0CC7800008D160020681500205416002088
S11366E08C1600206915002000B589B000A820216F
S11366F000F018FC00A93548FBF792FB002808D1EC
S11367000098002805D09DF80800C00601D4012097
S113671000E0002009B000BD2C48704780B52C482B
S1136720002180F824120A222A492948FAF764FF32
S1136730002803D12648012180F8241201BD10B598
S1136740234890F82402012802D12148FBF77FFA5C
S1136750FDF749F810F164041F4800F0B5FB012867
S113676003D1FDF740F88442F6D21848FBF782FBC8
S113677010BD80B5164890F82402012802D11448AF
S1136780FBF765FA01BD10B50400114890F8240226
S1136790012817D10E492000FBF71DFC002811D554
S11367A00B48002180F824120948FBF750FA09E04D
S11367B02178094800F072FB074800F044FB0028E8
S11367C0FAD0641C20780028F2D110BD3C7B000074
S11367D0A00A0020FC7B000000C0004080B500F04F
S11367E0A4FB02BD30380A2801D2012000E00020B9
S11367F0C0B2704772B6704762B67047DFF83804AB
S11368005FF0FF310160DFF834045FF0FF310160B5
S1136810704770B504000D001600200000F0A8F9C0
S1136820FF2805D02819401E00F0A2F9FF2801D145
S1136830002017E0600A4FF400714843DFF80014A9
S11368400968884207D12B0032002100DFF8EC03ED
S113685000F0E4F806E02B0032002100DFF8D80352
S113686000F0DCF870BD70B504000D00200000F0ED
S11368707FF906002819401E00F07AF9F6B2FF2EBF
S113688002D0C0B2FF2801D1002005E00100C9B246
S11368903000C0B200F02FF970BD80B50020009028
S11368A0DFF89803006810F1010F01D1012036E0F0
S11368B00098DFF888134968081800900098DFF8FA
S11368C07C138968081800900098DFF87013C96871
S11368D0081800900098DFF86413096908180090FC
S11368E00098DFF858134969081800900098DFF8F9
S11368F04C138969081800900098DFF84013C9699F
S1136900081800900098C04300900098401C009024
S113691000AA0421CA480068F030FFF77AFF02BDDC
S11369200020C749096809680818C5490968496801
S11369300818C349096889680818C1490968C968F9
S11369400818BF49096809690818BD4909684969EF
S11369500818BB49096889690818B9490968D1F850
S1136960F0100818002801D1012000E00020704731
S113697080B5B248006810F1010F06D0AF4800F0AE
S113698090F8002801D100200CE0AB48006810F119
S1136990010F06D0A84800F084F8002801D1002097
S11369A000E0012002BDA6480068704780B54FF49E
S11369B00072B1FBF2F303FB1213002B01D0002091
S11369C00BE002688A4201D1012006E001604FF425
S11369D00072001DFFF79EFD012002BD38B50400C2
S11369E00D009648844208D1934C29002000FFF7FB
S11369F0DDFF002810D100200FE091480068854297
S1136A0003D18E4C8E480568EFE7200000F049F86A
S1136A100028EAD1002000E0200032BD2DE9F04139
S1136A2004000F0015001E00780A4FF4007101FBEA
S1136A3000F8206810F1010F07D141462000FFF74C
S1136A40B5FF002801D1002029E02068404508D086
S1136A5041462000FFF7C2FF0400002C01D10020B2
S1136A601DE02068381A0019071DFCF7D0FE201D10
S1136A70381AB0F5007F0AD318F500712000FFF72B
S1136A80ADFF0400002C01D1002008E0271D287868
S1136A9038707F1C6D1C761E002EE6D10120BDE8E7
S1136AA0F081F8B505000124286800F061F8C0B24F
S1136AB0FF2801D100201DE0002600E0761C802E76
S1136AC016D2286810EB860715EB86004068009004
S1136AD0FCF79DFE0422390000A8FFF70AF80028FD
S1136AE001D0002404E0386800998842E6D00024EC
S1136AF02000C0B2F2BD70B50D00EDB2C0B2854247
S1136B0001D2002033E04E49097AC0B2884205D34D
S1136B104B4991F8BC10EDB2A94201D2002026E005
S1136B20C0B200F04FF804002800C0B200F04AF8E8
S1136B3006002800C0B200F062F88019401E001B55
S1136B40401C850A002600E0761CB6B2ADB2AE4207
S1136B500CD2FCF75CFEB6B24FF4806000FB06403A
S1136B60FEF7A0FF0028EFD0002000E0012070BD58
S1136B7038B50400002500E06D1CEDB2102D1FD2C5
S1136B80FCF745FEEDB20C202D4900FB0510006812
S1136B908442F1D3EDB20C20294900FB05100068B2
S1136BA0EDB20C21264A01FB0521496808188442EC
S1136BB0E2D2EDB20C20224900FB0510007A00E07D
S1136BC0FF2032BD38B50400002500E06D1CEDB295
S1136BD0102D11D2FCF71BFEEDB20C20184900FB5E
S1136BE00510007AE4B2A042F0D1EDB20C201449B1
S1136BF000FB0510006801E05FF0FF3032BD38B5DE
S1136C000400002500E06D1CEDB2102D11D2FCF73C
S1136C10FEFDEDB20C200A4900FB0510007AE4B237
S1136C20A042F0D1EDB20C20054900FB05104068EC
S1136C3000E0002032BD0000C80C0020CC0E002073
S1136C404474000062F30F2262F31F42401810F0F4
S1136C50030308D0C91A1FD3DB0748BF00F8012D6E
S1136C6028BF20F8022D130030B4144615461039FD
S1136C7028BF20E93C00FAD8490728BF20E90C00C6
S1136C8048BF40F8042D890028BF20F8022D48BFD2
S1136C9000F8012D30BC7047C91818BF00F8012D49
S1136CA0CB0728BF00F8012D70470000DFF83C1225
S1136CB088421BD0DFF83812884217D0DFF834122C
S1136CC0884213D0DFF8301288420FD0DFF82C123C
S1136CD088420BD0DFF82812884207D0DFF824124C
S1136CE0884203D0DFF82012884201D1012000E05D
S1136CF00020C0B27047F8B504000E0017001D0054
S1136D002000FFF7D3FF002805D14FF4B071DFF85E
S1136D10FC01FCF777FD002F05D140F26111DFF88B
S1136D20EC01FCF76FFDDFF8E801006810F0E04FBC
S1136D3027D0DFF8DC010068DFF8D8110840B0F193
S1136D40805F1ED0DFF8C8010068DFF8C811084072
S1136D50DFF8C411884205D1DFF8B401006880B2BD
S1136D6002280ED0DFF8A8010068DFF8A811084057
S1136D70DFF8A811884206D1DFF894010068000406
S1136D8001D1102000E0082000FB07F0864205D264
S1136D904FF4B171DFF87401FCF734FD200000F00A
S1136DA038F8B6EB071F05D2206B50F020002063A3
S1136DB07F0803E0206B30F020002063F000B0FB7C
S1136DC0F7F0401C4008810961624021B0FBF1F2F8
S1136DD002FB1102A262E5620020A061200000F023
S1136DE001F8F1BD10B504002000FFF75FFF002893
S1136DF005D14FF4FB71DFF81401FCF703FDE06AE1
S1136E0050F01000E062206B40F20131084320632F
S1136E1010BD10B504002000FFF748FF002805D17D
S1136E2040F21621DFF8E400FCF7ECFCA06900074F
S1136E30FCD4E06A30F01000E062206BDFF8E01070
S1136E400840206310BD10B504002000FFF72EFF9A
S1136E50002805D140F25541DFF8B000FCF7D2FC20
S1136E60A069C0F3401010F0010090F00100C0B21E
S1136E7010BD10B504002000FFF718FF002805D14D
S1136E8040F27641DFF88400FCF7BCFCA069C00640
S1136E9001D4206801E05FF0FF3010BD38B5040074
S1136EA00D002000FFF702FF002804D140F2C94181
S1136EB01648FCF7A7FCA069800603D4EDB2256050
S1136EC0012000E0002032BD10B504002000FFF7CF
S1136ED0EDFE002804D140F23B510C48FCF792FC33
S1136EE0A069C0F3C00010F0010010BD00C0004054
S1136EF000D0004000E0004000F0004000000140ED
S1136F0000100140002001400030014010770000D3
S1136F1000E00F400000FF700000011000000310AB
S1136F20FEFCFFFF002200F00BB810B504002000A7
S1136F3000F01FF8002801D0203CFFE7200010BD1E
S1136F4000B500BF130096469446103928BFA0E848
S1136F500C50FAD85FEA417C28BF0CC048BF40F807
S1136F60042BC90728BF20F8022B48BF00F8012BC7
S1136F7000BD61381A2801D2012000E00020C0B20F
S1136F8070470000610062006300640065006600F1
S1136F906700680069006A006B006C006D006E0099
S1136FA06F00700071007200730074007500760049
S1136FB07700780079007A00A100A200A300A50060
S1136FC0AC00AF00E000E100E200E300E400E50013
S1136FD0E600E700E800E900EA00EB00EC00ED0061
S1136FE0EE00EF00F000F100F200F300F400F50011
S1136FF0F600F800F900FA00FB00FC00FD00FE00BA
S1137000FF00010103010501070109010B010D0145
S11370100F01110113011501170119011B011D01B4
S11370201F01210123012501270129012B012D0124
S11370302F0131013301350137013A013C013E0191
S1137040400142014401460148014B014D014F01F9
S1137050510153015501570159015B015D015F0164
S1137060610163016501670169016B016D016F01D4
S113707071017301750177017A017C017E0192012E
S1137080B103B203B303B403B503B603B703B80340
S1137090B903BA03BB03BC03BD03BE03BF03C003F0
S11370A0C103C303C403C503C603C703C803C90399
S11370B0CA0330043104320433043404350436047E
S11370C03704380439043A043B043C043D043E04C8
S11370D03F04400441044204430444044504460478
S11370E04704480449044A044B044C044D044E0428
S11370F04F045104520453045404550456045704D1
S1137100580459045A045B045C045E045F0470214F
S113711071217221732174217521762177217821BF
S113712079217A217B217C217D217E217F2141FFD0
S113713042FF43FF44FF45FF46FF47FF48FF49FF27
S11371404AFF4BFF4CFF4DFF4EFF4FFF50FF51FFD7
S113715052FF53FF54FF55FF56FF57FF58FF59FF87
S11371605AFF00004100420043004400450046002D
S11371704700480049004A004B004C004D004E00B7
S11371804F00500051005200530054005500560067
S11371905700580059005A002100E0FFE1FFE5FFC5
S11371A0E2FFE3FFC000C100C200C300C400C50089
S11371B0C600C700C800C900CA00CB00CC00CD007F
S11371C0CE00CF00D000D100D200D300D400D5002F
S11371D0D600D800D900DA00DB00DC00DD00DE00D8
S11371E07801000102010401060108010A010C01F1
S11371F00E01100112011401160118011A011C01DB
S11372001E01200122012401260128012A012C014A
S11372102E01300132013401360139013B013D01B7
S11372203F0141014301450147014A014C014E011F
S1137230500152015401560158015A015C015E018A
S1137240600162016401660168016A016C016E01FA
S1137250700172017401760179017B017D01910154
S1137260910392039303940395039603970398035E
S113727099039A039B039C039D039E039F03A0030E
S1137280A103A303A403A503A603A703A803A903B7
S1137290AA0310041104120413041404150416049C
S11372A01704180419041A041B041C041D041E04E6
S11372B01F04200421042204230424042504260496
S11372C02704280429042A042B042C042D042E0446
S11372D02F0401040204030404040504060407043F
S11372E0080409040A040B040C040E040F046021AE
S11372F0612162216321642165216621672168215E
S113730069216A216B216C216D216E216F2121FF7E
S113731022FF23FF24FF25FF26FF27FF28FF29FF45
S11373202AFF2BFF2CFF2DFF2EFF2FFF30FF31FFF5
S113733032FF33FF34FF35FF36FF37FF38FF39FFA5
S11373403AFF0000C700FC00E900E200E400E000AE
S1137350E500E700EA00EB00E800EF00EE00EC00D7
S1137360C400C500C900E600C600F400F600F2003F
S1137370FB00F900FF00D600DC00A200A300A5007A
S1137380A7209201E100ED00F300FA00F100D10022
S1137390AA00BA00BF001023AC00BD00BC00A100CD
S11373A0AB00BB0091259225932502252425612558
S11373B06225562555256325512557255D255C25D0
S11373C05B251025142534252C251C2500253C255A
S11373D05E255F255A255425692566256025502597
S11373E06C2567256825642565255925582552256A
S11373F053256B256A2518250C25882584258C257D
S113740090258025B103DF009303C003A303C303C6
S1137410B500C403A6039803A903B4031E22C6033C
S1137420B50329226122B10065226422202321238D
S1137430F7004822B0001922B7001A227F20B200B8
S1137440A025A0000080000000200000040000002F
S113745000A00000002000000500000000C00000A3
S1137460002000000600000000E0000000200000F2
S113747007000000000001000020000008000000D8
S1137480002001000020000009000000004001006D
S1137490002000000A00000000600100002000003D
S11374A00B00000000800100002000000C00000020
S11374B000A00100002000000D00000000C0010039
S11374C0002000000E00000000E001000020000089
S11374D00F00000000000200008000001000000007
S11374E00080020000800000110000000000030082
S11374F000800000120000000080030000800000F3
S113750013000000809A90418E418F804545454983
S113751049498E8F9092924F994F555559999A9BFC
S11375209C9D9E9F41494F55A5A5A6A7A8A9AAAB76
S1137530AC21AEAFB0B1B2B3B4B5B6B7B8B9BABB9B
S1137540BCBDBEBFC0C1C2C3C4C5C6C7C8C9CACBFF
S1137550CCCDCECFD0D1D2D3D4D5D6D7D8D9DADBEF
S1137560DCDDDEDFE0E1E2E3E4E5E6E7E8E9EAEBDF
S1137570ECEDEEEFF0F1F2F3F4F5F6F7F8F9FAFBCF
S1137580FCFDFEFF40420F0000201C0080841E0012
S113759000802500999E36000040380000093D0017
S11375A000803E0000004B00404B4C0000204E0089
S11375B0808D5B0000C05D000080700000127A00C6
S11375C000007D0080969800001BB7000080BB007F
S11375D0C0E8CE00647ADA000024F4000000FA0067
S11375E080A81201002D310100366E0140787D0122
S11375F0433A5C576F726B5C736F66747761726544
S11376005C4F70656E424C545C5461726765745C87
S113761044656D6F5C41524D434D335F4C4D335364
S11376205F454B5F4C4D3353363936355F494152D4
S11376305C426F6F745C6C69625C647269766572DB
S11376406C69625C65746865726E65742E630000B3
S1137650433A5C576F726B5C736F667477617265E3
S11376605C4F70656E424C545C5461726765745C27
S113767044656D6F5C41524D434D335F4C4D335304
S11376805F454B5F4C4D3353363936355F49415274
S11376905C426F6F745C6C69625C6472697665727B
S11376A06C69625C666C6173686C69622E6300006D
S11376B0433A5C576F726B5C736F66747761726583
S11376C05C4F70656E424C545C5461726765745CC7
S11376D044656D6F5C41524D434D335F4C4D3353A4
S11376E05F454B5F4C4D3353363936355F49415214
S11376F05C426F6F745C6C69625C6472697665721B
S11377006C69625C73797363746C2E6300000000AF
S1137710433A5C576F726B5C736F66747761726522
S11377205C4F70656E424C545C5461726765745C66
S113773044656D6F5C41524D434D335F4C4D335343
S11377405F454B5F4C4D3353363936355F494152B3
S11377505C426F6F745C6C69625C647269766572BA
S11377606C69625C756172746C69622E63000000FE
S113777080B5154801210170FCF735F813490860FC
S113778000F001F801BD80B5FEF7D0FA012819D048
S1137790FEF7E3FA002815D00B480078012811D130
S11377A0FCF721F80949096801F51C511031884298
S11377B008D3054800210170FEF7D8FA002801D14A
S11377C0FEF78EFE01BD00008A1600203C16002044
S11377D0433A5C576F726B5C736F66747761726562
S11377E05C4F70656E424C545C5461726765745CA6
S11377F044656D6F5C41524D434D335F4C4D335383
S11378005F454B5F4C4D3353363936355F494152F2
S11378105C426F6F745C6C69625C647269766572F9
S11378206C69625C6770696F2E630000433A5C5751
S11378306F726B5C736F6674776172655C4F7065B1
S11378406E424C545C5461726765745C44656D6F40
S11378505C41524D434D335F4C4D33535F454B5F59
S11378604C4D3353363936355F4941525C426F6F64
S1137870745C6C69625C6472697665726C69625C82
S11378807373692E63000000433A5C576F726B5C3C
S1137890736F6674776172655C4F70656E424C54A9
S11378A05C5461726765745C536F757263655C41A7
S11378B0524D434D335F4C4D33535C4941525C76DA
S11378C06563746F72732E6300000000433A5C5763
S11378D06F726B5C736F6674776172655C4F706511
S11378E06E424C545C5461726765745C536F75727C
S11378F063655C41524D434D335F4C4D33535C756E
S11379006172742E6300000080B5FEF7E5FDFBF79D
S11379107DFFFBF749FFFEF70EFEFEF70BFAFEF7BD
S113792097F9FFF725FF01BD80B5FBF770FFFBF763
S113793050FFFEF735FAFEF799F9FFF724FF01BD72
S113794080B500F005F8FFF7DFFFFFF7EDFFFCE778
S113795080B50648FBF7F0FC0548FBF774FC0321EF
S11379605FF04020FBF79EF901BD00008003C001D9
S113797001000020433A5C576F726B5C736F66744E
S1137980776172655C4F70656E424C545C546172F1
S11379906765745C536F757263655C66696C652EAC
S11379A06300000050617273696E67206669726DCE
S11379B0776172652066696C6520746F206F6274EC
S11379C061696E2065726173652073697A652E2E14
S11379D02E0000004669726D7761726520757064CF
S11379E0617465207375636365737366756C6C7914
S11379F020636F6D706C657465640A0D000000008F
S1137A004F70656E696E67206669726D7761726525
S1137A102066696C6520666F722072656164696EA8
S1137A20672E2E2E0000000010B507497944183146
S1137A30064C7C44163404E00A68081D5118884733
S1137A400146A142F8D110BD98000000B800000022
S1137A504669726D77617265207570646174652022
S1137A6072657175657374206465746563746564A7
S1137A700A0D00005374617274696E67207468653E
S1137A802070726F6772616D6D696E6720736571C6
S1137A9075656E63650A0D0052656164696E6720E1
S1137AA06C696E652066726F6D2066696C652E2E3A
S1137AB02E4552524F520A0D00000000496E766165
S1137AC06C696420636865636B73756D20666F759C
S1137AD06E642E2E2E4552524F520A0D00000000A5
S1137AE093D1FFFF94160000040000200000000062
S1137AF013A5FFFF04000000900100000000002017
S1137B00000000002062797465732066726F6D2036
S1137B106D656D6F7279206174203078000000000B
S1137B2057726974696E672070726F6772616D2035
S1137B30636865636B73756D2E2E2E002F64656DFF
S1137B406F70726F675F656B5F6C6D337336393658
S1137B50352E737265630000206279746573207436
S1137B606F206D656D6F727920617420307800002C
S1137B70436C6F73696E67206669726D77617265B5
S1137B802066696C650A0D0000F009F8002801D030
S1137B90FFF74AFF0020FFF7D3FE00F002F80120B0
S1137BA0704700F001B800000746384600F002F8BC
S1137BB0FBE7000080B5C046C046024A1100182009
S1137BC0ABBEFBE726000200034B9D46C046C04601
S1137BD0C046C046FFF7D8FF9818002001030507E8
S1137BE0090E10121416181C1E00000050726F6744
S1137BF072616D6D696E6720000000002F626F6F07
S1137C00746C6F672E7478740000000080B53C219A
S1137C100148FBF7F7FD01BD88780000222A3A3CB1
S1137C203E3F7C7F0000000045726173696E6720EF
S1137C300000000040E00F4044E00F4048E00F40E7
S1137C4000E10F4004E10F4008E10F40C046C04688
S1137C50C046C046FFF798FF2B2C3B3D5B5D000000
S1137C604552524F520A0D004F4B0A0D00000000BE
S1137C70FFFFFFFFFFFF00004F70656E424C540092
S10F7C8000000000FFFFFFFF04010000F3
S9037C4D33
